 jaccessinspector-32

 Timestamp is ffffffff (Sun Feb  7 06:28:15 2106)

 Preferred load address is 00400000

 Start         Length     Name                   Class
 0001:00000000 00000020H .text$di                CODE
 0001:00000020 0000ca20H .text$mn                CODE
 0001:0000ca40 00000140H .text$x                 CODE
 0001:0000cb80 0000000fH .text$yd                CODE
 0002:00000000 00000220H .idata$5                DATA
 0002:00000220 00000004H .00cfg                  DATA
 0002:00000224 00000004H .CRT$XCA                DATA
 0002:00000228 00000004H .CRT$XCAA               DATA
 0002:0000022c 00000004H .CRT$XCU                DATA
 0002:00000230 00000004H .CRT$XCZ                DATA
 0002:00000234 00000004H .CRT$XIA                DATA
 0002:00000238 00000004H .CRT$XIAA               DATA
 0002:0000023c 00000004H .CRT$XIAC               DATA
 0002:00000240 00000004H .CRT$XIC                DATA
 0002:00000244 00000004H .CRT$XIZ                DATA
 0002:00000248 00000004H .CRT$XLA                DATA
 0002:0000024c 00000004H .CRT$XLZ                DATA
 0002:00000250 00000004H .CRT$XPA                DATA
 0002:00000254 00000004H .CRT$XPZ                DATA
 0002:00000258 00000004H .CRT$XTA                DATA
 0002:0000025c 00000004H .CRT$XTZ                DATA
 0002:00000260 00000000H .gfids$y                DATA
 0002:00000260 00002120H .rdata                  DATA
 0002:00002380 00000018H .rdata$T                DATA
 0002:00002398 00000138H .rdata$r                DATA
 0002:000024d0 00000028H .rdata$sxdata           DATA
 0002:000024f8 000003b0H .rdata$zzzdbg           DATA
 0002:000028a8 00000004H .rtc$IAA                DATA
 0002:000028ac 00000004H .rtc$IZZ                DATA
 0002:000028b0 00000004H .rtc$TAA                DATA
 0002:000028b4 00000004H .rtc$TZZ                DATA
 0002:000028b8 00000004H .tls                    DATA
 0002:000028bc 00000004H .tls$                   DATA
 0002:000028c0 00000008H .tls$ZZZ                DATA
 0002:000028c8 00000224H .xdata$x                DATA
 0002:00002aec 00000000H .edata                  DATA
 0002:00002aec 00000104H .idata$2                DATA
 0002:00002bf0 00000014H .idata$3                DATA
 0002:00002c04 00000220H .idata$4                DATA
 0002:00002e24 00000a00H .idata$6                DATA
 0003:00000000 00000ab8H .data                   DATA
 0003:00000ab8 00000088H .data$r                 DATA
 0003:00000b40 00000750H .bss                    DATA
 0004:00000000 000001c0H .rsrc$01                DATA
 0004:000001c0 00000ec0H .rsrc$02                DATA

  Address         Publics by Value              Rva+Base       Lib:Object

 0000:00000000       ___guard_fids_count        00000000     <absolute>
 0000:00000000       ___guard_iat_table         00000000     <absolute>
 0000:00000000       ___hybrid_code_map_count   00000000     <absolute>
 0000:00000000       ___enclave_config          00000000     <absolute>
 0000:00000000       ___guard_iat_count         00000000     <absolute>
 0000:00000000       ___dynamic_value_reloc_table 00000000     <absolute>
 0000:00000000       ___guard_longjmp_count     00000000     <absolute>
 0000:00000000       ___hybrid_code_map         00000000     <absolute>
 0000:00000000       ___guard_fids_table        00000000     <absolute>
 0000:00000000       ___volatile_metadata       00000000     <absolute>
 0000:00000000       ___hybrid_auxiliary_iat    00000000     <absolute>
 0000:00000000       ___guard_longjmp_table     00000000     <absolute>
 0000:0000000a       ___safe_se_handler_count   0000000a     <absolute>
 0000:0000002c       __tls_array                0000002c     <absolute>
 0000:00000100       ___guard_flags             00000100     <absolute>
 0000:00000000       ___ImageBase               00400000     <linker-defined>
 0001:00000020       _initializeAccessBridge    00401020 f   AccessBridgeCalls.obj
 0001:00000ee0       _shutdownAccessBridge      00401ee0 f   AccessBridgeCalls.obj
 0001:00000f30       _IsJavaWindow              00401f30 f   AccessBridgeCalls.obj
 0001:00000f60       _GetAccessibleContextFromHWND 00401f60 f   AccessBridgeCalls.obj
 0001:00000f90       _getHWNDFromAccessibleContext 00401f90 f   AccessBridgeCalls.obj
 0001:00000fc0       _SetJavaShutdown           00401fc0 f   AccessBridgeCalls.obj
 0001:00000fe0       _SetFocusGained            00401fe0 f   AccessBridgeCalls.obj
 0001:00001000       _SetFocusLost              00402000 f   AccessBridgeCalls.obj
 0001:00001020       _SetCaretUpdate            00402020 f   AccessBridgeCalls.obj
 0001:00001040       _SetMouseClicked           00402040 f   AccessBridgeCalls.obj
 0001:00001060       _SetMouseEntered           00402060 f   AccessBridgeCalls.obj
 0001:00001080       _SetMouseExited            00402080 f   AccessBridgeCalls.obj
 0001:000010a0       _SetMousePressed           004020a0 f   AccessBridgeCalls.obj
 0001:000010c0       _SetMouseReleased          004020c0 f   AccessBridgeCalls.obj
 0001:000010e0       _SetMenuCanceled           004020e0 f   AccessBridgeCalls.obj
 0001:00001100       _SetMenuDeselected         00402100 f   AccessBridgeCalls.obj
 0001:00001120       _SetMenuSelected           00402120 f   AccessBridgeCalls.obj
 0001:00001140       _SetPopupMenuCanceled      00402140 f   AccessBridgeCalls.obj
 0001:00001160       _SetPopupMenuWillBecomeInvisible 00402160 f   AccessBridgeCalls.obj
 0001:00001180       _SetPopupMenuWillBecomeVisible 00402180 f   AccessBridgeCalls.obj
 0001:000011a0       _SetPropertyNameChange     004021a0 f   AccessBridgeCalls.obj
 0001:000011c0       _SetPropertyDescriptionChange 004021c0 f   AccessBridgeCalls.obj
 0001:000011e0       _SetPropertyStateChange    004021e0 f   AccessBridgeCalls.obj
 0001:00001200       _SetPropertyValueChange    00402200 f   AccessBridgeCalls.obj
 0001:00001220       _SetPropertySelectionChange 00402220 f   AccessBridgeCalls.obj
 0001:00001240       _SetPropertyTextChange     00402240 f   AccessBridgeCalls.obj
 0001:00001260       _SetPropertyCaretChange    00402260 f   AccessBridgeCalls.obj
 0001:00001280       _SetPropertyVisibleDataChange 00402280 f   AccessBridgeCalls.obj
 0001:000012a0       _SetPropertyChildChange    004022a0 f   AccessBridgeCalls.obj
 0001:000012c0       _SetPropertyActiveDescendentChange 004022c0 f   AccessBridgeCalls.obj
 0001:000012e0       _SetPropertyTableModelChange 004022e0 f   AccessBridgeCalls.obj
 0001:00001300       _ReleaseJavaObject         00402300 f   AccessBridgeCalls.obj
 0001:00001330       _GetVersionInfo            00402330 f   AccessBridgeCalls.obj
 0001:00001360       _GetAccessibleContextAt    00402360 f   AccessBridgeCalls.obj
 0001:000013a0       _GetAccessibleContextWithFocus 004023a0 f   AccessBridgeCalls.obj
 0001:000013d0       _GetAccessibleContextInfo  004023d0 f   AccessBridgeCalls.obj
 0001:00001400       _GetAccessibleChildFromContext 00402400 f   AccessBridgeCalls.obj
 0001:00001430       _GetAccessibleParentFromContext 00402430 f   AccessBridgeCalls.obj
 0001:00001460       _GetAccessibleTextInfo     00402460 f   AccessBridgeCalls.obj
 0001:000014a0       _GetAccessibleTextItems    004024a0 f   AccessBridgeCalls.obj
 0001:000014d0       _GetAccessibleTextSelectionInfo 004024d0 f   AccessBridgeCalls.obj
 0001:00001500       _GetAccessibleTextAttributes 00402500 f   AccessBridgeCalls.obj
 0001:00001530       _GetAccessibleTextRect     00402530 f   AccessBridgeCalls.obj
 0001:00001560       _GetAccessibleTextLineBounds 00402560 f   AccessBridgeCalls.obj
 0001:000015a0       _GetAccessibleTextRange    004025a0 f   AccessBridgeCalls.obj
 0001:000015e0       _getAccessibleTableInfo    004025e0 f   AccessBridgeCalls.obj
 0001:00001610       _getAccessibleTableCellInfo 00402610 f   AccessBridgeCalls.obj
 0001:00001650       _getAccessibleTableRowHeader 00402650 f   AccessBridgeCalls.obj
 0001:00001680       _getAccessibleTableColumnHeader 00402680 f   AccessBridgeCalls.obj
 0001:000016b0       _getAccessibleTableRowDescription 004026b0 f   AccessBridgeCalls.obj
 0001:000016e0       _getAccessibleTableColumnDescription 004026e0 f   AccessBridgeCalls.obj
 0001:00001710       _getAccessibleTableRowSelectionCount 00402710 f   AccessBridgeCalls.obj
 0001:00001740       _isAccessibleTableRowSelected 00402740 f   AccessBridgeCalls.obj
 0001:00001770       _getAccessibleTableRowSelections 00402770 f   AccessBridgeCalls.obj
 0001:000017a0       _getAccessibleTableColumnSelectionCount 004027a0 f   AccessBridgeCalls.obj
 0001:000017d0       _isAccessibleTableColumnSelected 004027d0 f   AccessBridgeCalls.obj
 0001:00001800       _getAccessibleTableColumnSelections 00402800 f   AccessBridgeCalls.obj
 0001:00001830       _getAccessibleTableRow     00402830 f   AccessBridgeCalls.obj
 0001:00001860       _getAccessibleTableColumn  00402860 f   AccessBridgeCalls.obj
 0001:00001890       _getAccessibleTableIndex   00402890 f   AccessBridgeCalls.obj
 0001:000018c0       _getAccessibleRelationSet  004028c0 f   AccessBridgeCalls.obj
 0001:000018f0       _getAccessibleHypertext    004028f0 f   AccessBridgeCalls.obj
 0001:00001920       _activateAccessibleHyperlink 00402920 f   AccessBridgeCalls.obj
 0001:00001950       _getAccessibleHyperlinkCount 00402950 f   AccessBridgeCalls.obj
 0001:00001980       _getAccessibleHypertextExt 00402980 f   AccessBridgeCalls.obj
 0001:000019b0       _getAccessibleHypertextLinkIndex 004029b0 f   AccessBridgeCalls.obj
 0001:000019e0       _getAccessibleHyperlink    004029e0 f   AccessBridgeCalls.obj
 0001:00001a10       _getAccessibleKeyBindings  00402a10 f   AccessBridgeCalls.obj
 0001:00001a40       _getAccessibleIcons        00402a40 f   AccessBridgeCalls.obj
 0001:00001a70       _getAccessibleActions      00402a70 f   AccessBridgeCalls.obj
 0001:00001aa0       _doAccessibleActions       00402aa0 f   AccessBridgeCalls.obj
 0001:00001ad0       _IsSameObject              00402ad0 f   AccessBridgeCalls.obj
 0001:00001b00       _setTextContents           00402b00 f   AccessBridgeCalls.obj
 0001:00001b30       _getParentWithRole         00402b30 f   AccessBridgeCalls.obj
 0001:00001b60       _getParentWithRoleElseRoot 00402b60 f   AccessBridgeCalls.obj
 0001:00001b90       _getTopLevelObject         00402b90 f   AccessBridgeCalls.obj
 0001:00001bc0       _getObjectDepth            00402bc0 f   AccessBridgeCalls.obj
 0001:00001bf0       _getActiveDescendent       00402bf0 f   AccessBridgeCalls.obj
 0001:00001c20       _GetCurrentAccessibleValueFromContext 00402c20 f   AccessBridgeCalls.obj
 0001:00001c50       _GetMaximumAccessibleValueFromContext 00402c50 f   AccessBridgeCalls.obj
 0001:00001c80       _GetMinimumAccessibleValueFromContext 00402c80 f   AccessBridgeCalls.obj
 0001:00001cb0       _GetAccessibleSelectionFromContext 00402cb0 f   AccessBridgeCalls.obj
 0001:00001ce0       _GetAccessibleSelectionCountFromContext 00402ce0 f   AccessBridgeCalls.obj
 0001:00001d10       _IsAccessibleChildSelectedFromContext 00402d10 f   AccessBridgeCalls.obj
 0001:00001d40       _RemoveAccessibleSelectionFromContext 00402d40 f   AccessBridgeCalls.obj
 0001:00001d70       _SelectAllAccessibleSelectionFromContext 00402d70 f   AccessBridgeCalls.obj
 0001:00001da0       _getVirtualAccessibleName  00402da0 f   AccessBridgeCalls.obj
 0001:00001dd0       _requestFocus              00402dd0 f   AccessBridgeCalls.obj
 0001:00001e00       _selectTextRange           00402e00 f   AccessBridgeCalls.obj
 0001:00001e30       _getTextAttributesInRange  00402e30 f   AccessBridgeCalls.obj
 0001:00001e70       _getVisibleChildrenCount   00402e70 f   AccessBridgeCalls.obj
 0001:00001ea0       _getVisibleChildren        00402ea0 f   AccessBridgeCalls.obj
 0001:00001ed0       _setCaretPosition          00402ed0 f   AccessBridgeCalls.obj
 0001:00001f00       _getCaretLocation          00402f00 f   AccessBridgeCalls.obj
 0001:00001f30       _getEventsWaiting          00402f30 f   AccessBridgeCalls.obj
 0001:00001f50       _addAccessibleSelectionFromContext 00402f50 f   AccessBridgeCalls.obj
 0001:00001f80       _clearAccessibleSelectionFromContext 00402f80 f   AccessBridgeCalls.obj
 0001:00001fc0       _printError                00402fc0 f   AccessBridgeDebug.obj
 0001:000020d0       _PrintDebugString          004030d0 f   AccessBridgeDebug.obj
 0001:00002140       _wPrintJavaDebugString     00403140 f   AccessBridgeDebug.obj
 0001:000021b0       _wPrintDebugString         004031b0 f   AccessBridgeDebug.obj
 0001:00002220       _initializeFileLogger      00403220 f   AccessBridgeDebug.obj
 0001:00002350       _finalizeFileLogger        00403350 f   AccessBridgeDebug.obj
 0001:00002380       _getTimeStamp              00403380 f   AccessBridgeDebug.obj
 0001:000023c0       _PrintJavaDebugString2     004033c0 f   AccessBridgeDebug.obj
 0001:00002430       ___local_stdio_printf_options 00403430 f i AccessBridgeDebug.obj
 0001:00002440       __vfprintf_l               00403440 f i AccessBridgeDebug.obj
 0001:00002470       __vfwprintf_l              00403470 f i AccessBridgeDebug.obj
 0001:000024a0       _fprintf                   004034a0 f i AccessBridgeDebug.obj
 0001:000024e0       _printf                    004034e0 f i AccessBridgeDebug.obj
 0001:00002520       _vfprintf                  00403520 f i AccessBridgeDebug.obj
 0001:00002540       _vfwprintf                 00403540 f i AccessBridgeDebug.obj
 0001:00002560       ?initBroadcastMessageIDs@@YAHXZ 00403560 f   AccessBridgeMessages.obj
 0001:000025a0       ?getTimeAndDate@@YAPADXZ   004035a0 f   AccessInfo.obj
 0001:00002650       ?displayAndLog@@YAXPAUHWND__@@HPAU_iobuf@@PADZZ 00403650 f   AccessInfo.obj
 0001:00002730       ?logString@@YAXPAU_iobuf@@PADZZ 00403730 f   AccessInfo.obj
 0001:000027c0       ?getAccessibleInfo@@YAPADJ_JPADH@Z 004037c0 f   AccessInfo.obj
 0001:000027f0       ?getAccessibleInfo@@YAPADJ_JHHPADH@Z 004037f0 f   AccessInfo.obj
 0001:000049f0       ?appendToBuffer@@YAHPADI0ZZ 004059f0 f   AccessInfo.obj
 0001:00004ad0       __vsnprintf_l              00405ad0 f i AccessInfo.obj
 0001:00004b30       __vsprintf_l               00405b30 f i AccessInfo.obj
 0001:00004b50       _sprintf                   00405b50 f i AccessInfo.obj
 0001:00004b90       _vsprintf                  00405b90 f i AccessInfo.obj
 0001:00004bb0       ?AddMessage@MessageHistory@@QAEXPBD@Z 00405bb0 f   MessageHistory.obj
 0001:00004c80       ?GetFirstMessage@MessageHistory@@QAEPBDXZ 00405c80 f   MessageHistory.obj
 0001:00004cd0       ?GetPreviousMessage@MessageHistory@@QAEPBDXZ 00405cd0 f   MessageHistory.obj
 0001:00004d30       ?GetNextMessage@MessageHistory@@QAEPBDXZ 00405d30 f   MessageHistory.obj
 0001:00004da0       ?GetLastMessage@MessageHistory@@QAEPBDXZ 00405da0 f   MessageHistory.obj
 0001:00004e00       ?GetCurrentMessage@MessageHistory@@QAEPBDXZ 00405e00 f   MessageHistory.obj
 0001:00004e40       ?GetMessageA@MessageHistory@@QAEPBDI@Z 00405e40 f   MessageHistory.obj
 0001:00004ec0       ?GetCurrentMessageIndex@MessageHistory@@QAEIXZ 00405ec0 f   MessageHistory.obj
 0001:00004f10       ?IsFirstMessage@MessageHistory@@QAEHXZ 00405f10 f   MessageHistory.obj
 0001:00004f60       ?IsLastMessage@MessageHistory@@QAEHXZ 00405f60 f   MessageHistory.obj
 0001:00004fc0       ?GetMessageCount@MessageHistory@@QAEIXZ 00405fc0 f   MessageHistory.obj
 0001:00004fe0       ?clear@MessageHistory@@QAEXXZ 00405fe0 f   MessageHistory.obj
 0001:00005000       ??$?0$$V@?$_Compressed_pair@V?$allocator@D@std@@V?$_String_val@U?$_Simple_types@D@std@@@2@$00@std@@QAE@U_Zero_then_variadic_args_t@1@@Z 00406000 f i MessageHistory.obj
 0001:00005020       ??$?0V?$allocator@D@std@@$$V@?$_Compressed_pair@V?$allocator@D@std@@V?$_String_val@U?$_Simple_types@D@std@@@2@$00@std@@QAE@U_One_then_variadic_args_t@1@$$QAV?$allocator@D@1@@Z 00406020 f i MessageHistory.obj
 0001:00005050       ??$?0V?$allocator@D@std@@X@?$_String_alloc@U?$_String_base_types@DV?$allocator@D@std@@@std@@@std@@QAE@$$QAV?$allocator@D@1@@Z 00406050 f i MessageHistory.obj
 0001:00005080       ??$_Advance1@V?$_List_const_iterator@V?$_List_val@U?$_List_simple_types@V?$basic_string@DU?$char_traits@D@std@@V?$allocator@D@2@@std@@@std@@@std@@@std@@I@std@@YAXAAV?$_List_const_iterator@V?$_List_val@U?$_List_simple_types@V?$basic_string@DU?$char_traits@D@std@@V?$allocator@D@2@@std@@@std@@@std@@@0@IUbidirectional_iterator_tag@0@@Z 00406080 f i MessageHistory.obj
 0001:000050c0       ??$_Allocate@$07U_Default_allocate_traits@std@@$0A@@std@@YAPAXI@Z 004060c0 f i MessageHistory.obj
 0001:00005100       ??$_Allocate_manually_vector_aligned@U_Default_allocate_traits@std@@@std@@YAPAXI@Z 00406100 f i MessageHistory.obj
 0001:00005170       ??$_Buynode@V?$basic_string@DU?$char_traits@D@std@@V?$allocator@D@2@@std@@@?$_List_buy@V?$basic_string@DU?$char_traits@D@std@@V?$allocator@D@2@@std@@V?$allocator@V?$basic_string@DU?$char_traits@D@std@@V?$allocator@D@2@@std@@@2@@std@@QAEPAU?$_List_node@V?$basic_string@DU?$char_traits@D@std@@V?$allocator@D@2@@std@@PAX@1@PAU21@0$$QAV?$basic_string@DU?$char_traits@D@std@@V?$allocator@D@2@@1@@Z 00406170 f i MessageHistory.obj
 0001:00005240       ??$_Get_size_of_n@$00@std@@YAII@Z 00406240 f i MessageHistory.obj
 0001:00005240       ??$addressof@PAD@std@@YAPAPADAAPAD@Z 00406240 f i MessageHistory.obj
 0001:00005240       ??$_Unfancy@D@std@@YAPADPAD@Z 00406240 f i MessageHistory.obj
 0001:00005240       ??$forward@ABQAD@std@@YAABQADABQAD@Z 00406240 f i MessageHistory.obj
 0001:00005240       ??$_Convert_size@I@std@@YAII@Z 00406240 f i MessageHistory.obj
 0001:00005240       ??$forward@V?$basic_string@DU?$char_traits@D@std@@V?$allocator@D@2@@std@@@std@@YA$$QAV?$basic_string@DU?$char_traits@D@std@@V?$allocator@D@2@@0@AAV10@@Z 00406240 f i MessageHistory.obj
 0001:00005240       ??$addressof@PAU?$_List_node@V?$basic_string@DU?$char_traits@D@std@@V?$allocator@D@2@@std@@PAX@std@@@std@@YAPAPAU?$_List_node@V?$basic_string@DU?$char_traits@D@std@@V?$allocator@D@2@@std@@PAX@0@AAPAU10@@Z 00406240 f i MessageHistory.obj
 0001:00005240       ??$addressof@V?$_String_val@U?$_Simple_types@D@std@@@std@@@std@@YAPAV?$_String_val@U?$_Simple_types@D@std@@@0@AAV10@@Z 00406240 f i MessageHistory.obj
 0001:00005240       ??$addressof@V?$basic_string@DU?$char_traits@D@std@@V?$allocator@D@2@@std@@@std@@YAPAV?$basic_string@DU?$char_traits@D@std@@V?$allocator@D@2@@0@AAV10@@Z 00406240 f i MessageHistory.obj
 0001:00005240       ??$addressof@$$CBV?$_List_val@U?$_List_simple_types@V?$basic_string@DU?$char_traits@D@std@@V?$allocator@D@2@@std@@@std@@@std@@@std@@YAPBV?$_List_val@U?$_List_simple_types@V?$basic_string@DU?$char_traits@D@std@@V?$allocator@D@2@@std@@@std@@@0@ABV10@@Z 00406240 f i MessageHistory.obj
 0001:00005240       ??$addressof@V?$_List_val@U?$_List_simple_types@V?$basic_string@DU?$char_traits@D@std@@V?$allocator@D@2@@std@@@std@@@std@@@std@@YAPAV?$_List_val@U?$_List_simple_types@V?$basic_string@DU?$char_traits@D@std@@V?$allocator@D@2@@std@@@std@@@0@AAV10@@Z 00406240 f i MessageHistory.obj
 0001:00005240       ??$forward@V?$allocator@D@std@@@std@@YA$$QAV?$allocator@D@0@AAV10@@Z 00406240 f i MessageHistory.obj
 0001:00005240       ??$move@AAV?$basic_string@DU?$char_traits@D@std@@V?$allocator@D@2@@std@@@std@@YA$$QAV?$basic_string@DU?$char_traits@D@std@@V?$allocator@D@2@@0@AAV10@@Z 00406240 f i MessageHistory.obj
 0001:00005240       ??$forward@AAPAU?$_List_node@V?$basic_string@DU?$char_traits@D@std@@V?$allocator@D@2@@std@@PAX@std@@@std@@YAAAPAU?$_List_node@V?$basic_string@DU?$char_traits@D@std@@V?$allocator@D@2@@std@@PAX@0@AAPAU10@@Z 00406240 f i MessageHistory.obj
 0001:00005240       ??$move@AAV?$allocator@D@std@@@std@@YA$$QAV?$allocator@D@0@AAV10@@Z 00406240 f i MessageHistory.obj
 0001:00005250       ??$_Deallocate@$07$0A@@std@@YAXPAXI@Z 00406250 f i MessageHistory.obj
 0001:00005280       ??$_Distance1@V?$_List_const_iterator@V?$_List_val@U?$_List_simple_types@V?$basic_string@DU?$char_traits@D@std@@V?$allocator@D@2@@std@@@std@@@std@@@std@@@std@@YAHV?$_List_const_iterator@V?$_List_val@U?$_List_simple_types@V?$basic_string@DU?$char_traits@D@std@@V?$allocator@D@2@@std@@@std@@@std@@@0@0Uinput_iterator_tag@0@@Z 00406280 f i MessageHistory.obj
 0001:000052c0       ??$_Freenode0@V?$allocator@U?$_List_node@V?$basic_string@DU?$char_traits@D@std@@V?$allocator@D@2@@std@@PAX@std@@@std@@@?$_List_node@V?$basic_string@DU?$char_traits@D@std@@V?$allocator@D@2@@std@@PAX@std@@SAXAAV?$allocator@U?$_List_node@V?$basic_string@DU?$char_traits@D@std@@V?$allocator@D@2@@std@@PAX@std@@@1@PAU01@@Z 004062c0 f i MessageHistory.obj
 0001:00005340       ??$_Get_size_of_n@$0CA@@std@@YAII@Z 00406340 f i MessageHistory.obj
 0001:00005370       ??$_Insert@V?$basic_string@DU?$char_traits@D@std@@V?$allocator@D@2@@std@@@?$list@V?$basic_string@DU?$char_traits@D@std@@V?$allocator@D@2@@std@@V?$allocator@V?$basic_string@DU?$char_traits@D@std@@V?$allocator@D@2@@std@@@2@@std@@QAEXV?$_List_unchecked_const_iterator@V?$_List_val@U?$_List_simple_types@V?$basic_string@DU?$char_traits@D@std@@V?$allocator@D@2@@std@@@std@@@std@@U_Iterator_base0@2@@1@$$QAV?$basic_string@DU?$char_traits@D@std@@V?$allocator@D@2@@1@@Z 00406370 f i MessageHistory.obj
 0001:000053d0       ??$_Max_value@I@std@@YAABIABI0@Z 004063d0 f i MessageHistory.obj
 0001:00005400       ??$_Min_value@I@std@@YAABIABI0@Z 00406400 f i MessageHistory.obj
 0001:00005430       ??$_Reallocate_for@V<lambda_9366063389c5f42a00a5088cf24e69de>@@PBD@?$basic_string@DU?$char_traits@D@std@@V?$allocator@D@2@@std@@QAEAAV01@IV<lambda_9366063389c5f42a00a5088cf24e69de>@@PBD@Z 00406430 f i MessageHistory.obj
 0001:00005510       ??$advance@V?$_List_const_iterator@V?$_List_val@U?$_List_simple_types@V?$basic_string@DU?$char_traits@D@std@@V?$allocator@D@2@@std@@@std@@@std@@@std@@I@std@@YAXAAV?$_List_const_iterator@V?$_List_val@U?$_List_simple_types@V?$basic_string@DU?$char_traits@D@std@@V?$allocator@D@2@@std@@@std@@@std@@@0@I@Z 00406510 f i MessageHistory.obj
 0001:00005530       ??$construct@PAU?$_List_node@V?$basic_string@DU?$char_traits@D@std@@V?$allocator@D@2@@std@@PAX@std@@AAPAU12@@?$_Default_allocator_traits@V?$allocator@U?$_List_node@V?$basic_string@DU?$char_traits@D@std@@V?$allocator@D@2@@std@@PAX@std@@@std@@@std@@SAXAAV?$allocator@U?$_List_node@V?$basic_string@DU?$char_traits@D@std@@V?$allocator@D@2@@std@@PAX@std@@@1@QAPAU?$_List_node@V?$basic_string@DU?$char_traits@D@std@@V?$allocator@D@2@@std@@PAX@1@AAPAU31@@Z 00406530 f i MessageHistory.obj
 0001:00005530       ??$construct@PADABQAD@?$_Default_allocator_traits@V?$allocator@D@std@@@std@@SAXAAV?$allocator@D@1@QAPADABQAD@Z 00406530 f i MessageHistory.obj
 0001:00005560       ??$construct@V?$basic_string@DU?$char_traits@D@std@@V?$allocator@D@2@@std@@V12@@?$_Default_allocator_traits@V?$allocator@U?$_List_node@V?$basic_string@DU?$char_traits@D@std@@V?$allocator@D@2@@std@@PAX@std@@@std@@@std@@SAXAAV?$allocator@U?$_List_node@V?$basic_string@DU?$char_traits@D@std@@V?$allocator@D@2@@std@@PAX@std@@@1@QAV?$basic_string@DU?$char_traits@D@std@@V?$allocator@D@2@@1@$$QAV31@@Z 00406560 f i MessageHistory.obj
 0001:00005590       ??$destroy@PAD@?$_Default_allocator_traits@V?$allocator@D@std@@@std@@SAXAAV?$allocator@D@1@QAPAD@Z 00406590 f i MessageHistory.obj
 0001:00005590       ??$destroy@PAU?$_List_node@V?$basic_string@DU?$char_traits@D@std@@V?$allocator@D@2@@std@@PAX@std@@@?$_Default_allocator_traits@V?$allocator@U?$_List_node@V?$basic_string@DU?$char_traits@D@std@@V?$allocator@D@2@@std@@PAX@std@@@std@@@std@@SAXAAV?$allocator@U?$_List_node@V?$basic_string@DU?$char_traits@D@std@@V?$allocator@D@2@@std@@PAX@std@@@1@QAPAU?$_List_node@V?$basic_string@DU?$char_traits@D@std@@V?$allocator@D@2@@std@@PAX@1@@Z 00406590 f i MessageHistory.obj
 0001:000055a0       ??$destroy@V?$basic_string@DU?$char_traits@D@std@@V?$allocator@D@2@@std@@@?$_Default_allocator_traits@V?$allocator@U?$_List_node@V?$basic_string@DU?$char_traits@D@std@@V?$allocator@D@2@@std@@PAX@std@@@std@@@std@@SAXAAV?$allocator@U?$_List_node@V?$basic_string@DU?$char_traits@D@std@@V?$allocator@D@2@@std@@PAX@std@@@1@QAV?$basic_string@DU?$char_traits@D@std@@V?$allocator@D@2@@1@@Z 004065a0 f i MessageHistory.obj
 0001:000055b0       ??$distance@V?$_List_const_iterator@V?$_List_val@U?$_List_simple_types@V?$basic_string@DU?$char_traits@D@std@@V?$allocator@D@2@@std@@@std@@@std@@@std@@@std@@YAHV?$_List_const_iterator@V?$_List_val@U?$_List_simple_types@V?$basic_string@DU?$char_traits@D@std@@V?$allocator@D@2@@std@@@std@@@std@@@0@0@Z 004065b0 f i MessageHistory.obj
 0001:000055d0       ??0?$_List_const_iterator@V?$_List_val@U?$_List_simple_types@V?$basic_string@DU?$char_traits@D@std@@V?$allocator@D@2@@std@@@std@@@std@@@std@@QAE@PAU?$_List_node@V?$basic_string@DU?$char_traits@D@std@@V?$allocator@D@2@@std@@PAX@1@PBV?$_List_val@U?$_List_simple_types@V?$basic_string@DU?$char_traits@D@std@@V?$allocator@D@2@@std@@@std@@@1@@Z 004065d0 f i MessageHistory.obj
 0001:000055d0       ??0?$_List_unchecked_iterator@V?$_List_val@U?$_List_simple_types@V?$basic_string@DU?$char_traits@D@std@@V?$allocator@D@2@@std@@@std@@@std@@@std@@QAE@PAU?$_List_node@V?$basic_string@DU?$char_traits@D@std@@V?$allocator@D@2@@std@@PAX@1@PBV?$_List_val@U?$_List_simple_types@V?$basic_string@DU?$char_traits@D@std@@V?$allocator@D@2@@std@@@std@@@1@@Z 004065d0 f i MessageHistory.obj
 0001:000055f0       ??0?$_List_iterator@V?$_List_val@U?$_List_simple_types@V?$basic_string@DU?$char_traits@D@std@@V?$allocator@D@2@@std@@@std@@@std@@@std@@QAE@PAU?$_List_node@V?$basic_string@DU?$char_traits@D@std@@V?$allocator@D@2@@std@@PAX@1@PBV?$_List_val@U?$_List_simple_types@V?$basic_string@DU?$char_traits@D@std@@V?$allocator@D@2@@std@@@std@@@1@@Z 004065f0 f i MessageHistory.obj
 0001:00005610       ??0?$_List_unchecked_const_iterator@V?$_List_val@U?$_List_simple_types@V?$basic_string@DU?$char_traits@D@std@@V?$allocator@D@2@@std@@@std@@@std@@U_Iterator_base0@2@@std@@QAE@PAU?$_List_node@V?$basic_string@DU?$char_traits@D@std@@V?$allocator@D@2@@std@@PAX@1@PBV?$_List_val@U?$_List_simple_types@V?$basic_string@DU?$char_traits@D@std@@V?$allocator@D@2@@std@@@std@@@1@@Z 00406610 f i MessageHistory.obj
 0001:00005640       ??0?$_String_alloc@U?$_String_base_types@DV?$allocator@D@std@@@std@@@std@@QAE@XZ 00406640 f i MessageHistory.obj
 0001:00005660       ??0?$_String_val@U?$_Simple_types@D@std@@@std@@QAE@XZ 00406660 f i MessageHistory.obj
 0001:00005690       ??0?$allocator@D@std@@QAE@XZ 00406690 f i MessageHistory.obj
 0001:00005690       ?_Get_second@?$_Compressed_pair@V?$allocator@U?$_List_node@V?$basic_string@DU?$char_traits@D@std@@V?$allocator@D@2@@std@@PAX@std@@@std@@V?$_List_val@U?$_List_simple_types@V?$basic_string@DU?$char_traits@D@std@@V?$allocator@D@2@@std@@@std@@@2@$00@std@@QBEABV?$_List_val@U?$_List_simple_types@V?$basic_string@DU?$char_traits@D@std@@V?$allocator@D@2@@std@@@std@@@2@XZ 00406690 f i MessageHistory.obj
 0001:00005690       ?_Get_first@?$_Compressed_pair@V?$allocator@D@std@@V?$_String_val@U?$_Simple_types@D@std@@@2@$00@std@@QBEABV?$allocator@D@2@XZ 00406690 f i MessageHistory.obj
 0001:00005690       ?_Get_first@?$_Compressed_pair@V?$allocator@U?$_List_node@V?$basic_string@DU?$char_traits@D@std@@V?$allocator@D@2@@std@@PAX@std@@@std@@V?$_List_val@U?$_List_simple_types@V?$basic_string@DU?$char_traits@D@std@@V?$allocator@D@2@@std@@@std@@@2@$00@std@@QBEABV?$allocator@U?$_List_node@V?$basic_string@DU?$char_traits@D@std@@V?$allocator@D@2@@std@@PAX@std@@@2@XZ 00406690 f i MessageHistory.obj
 0001:00005690       ?_Get_second@?$_Compressed_pair@V?$allocator@D@std@@V?$_String_val@U?$_Simple_types@D@std@@@2@$00@std@@QBEABV?$_String_val@U?$_Simple_types@D@std@@@2@XZ 00406690 f i MessageHistory.obj
 0001:00005690       ?_Get_first@?$_Compressed_pair@V?$allocator@D@std@@V?$_String_val@U?$_Simple_types@D@std@@@2@$00@std@@QAEAAV?$allocator@D@2@XZ 00406690 f i MessageHistory.obj
 0001:00005690       ?_Get_second@?$_Compressed_pair@V?$allocator@D@std@@V?$_String_val@U?$_Simple_types@D@std@@@2@$00@std@@QAEAAV?$_String_val@U?$_Simple_types@D@std@@@2@XZ 00406690 f i MessageHistory.obj
 0001:00005690       ??0_Bxty@?$_String_val@U?$_Simple_types@D@std@@@std@@QAE@XZ 00406690 f i MessageHistory.obj
 0001:00005690       ?_Get_second@?$_Compressed_pair@V?$allocator@U?$_List_node@V?$basic_string@DU?$char_traits@D@std@@V?$allocator@D@2@@std@@PAX@std@@@std@@V?$_List_val@U?$_List_simple_types@V?$basic_string@DU?$char_traits@D@std@@V?$allocator@D@2@@std@@@std@@@2@$00@std@@QAEAAV?$_List_val@U?$_List_simple_types@V?$basic_string@DU?$char_traits@D@std@@V?$allocator@D@2@@std@@@std@@@2@XZ 00406690 f i MessageHistory.obj
 0001:00005690       ??0?$allocator@U?$_List_node@V?$basic_string@DU?$char_traits@D@std@@V?$allocator@D@2@@std@@PAX@std@@@std@@QAE@XZ 00406690 f i jaccessinspector.obj
 0001:00005690       ?_Get_first@?$_Compressed_pair@V?$allocator@U?$_List_node@V?$basic_string@DU?$char_traits@D@std@@V?$allocator@D@2@@std@@PAX@std@@@std@@V?$_List_val@U?$_List_simple_types@V?$basic_string@DU?$char_traits@D@std@@V?$allocator@D@2@@std@@@std@@@2@$00@std@@QAEAAV?$allocator@U?$_List_node@V?$basic_string@DU?$char_traits@D@std@@V?$allocator@D@2@@std@@PAX@std@@@2@XZ 00406690 f i MessageHistory.obj
 0001:000056a0       ??0?$basic_string@DU?$char_traits@D@std@@V?$allocator@D@2@@std@@QAE@$$QAV01@@Z 004066a0 f i MessageHistory.obj
 0001:00005720       ??0?$basic_string@DU?$char_traits@D@std@@V?$allocator@D@2@@std@@QAE@QBD@Z 00406720 f i MessageHistory.obj
 0001:00005790       ??1?$_Compressed_pair@V?$allocator@D@std@@V?$_String_val@U?$_Simple_types@D@std@@@2@$00@std@@QAE@XZ 00406790 f i MessageHistory.obj
 0001:000057b0       ??1?$_String_alloc@U?$_String_base_types@DV?$allocator@D@std@@@std@@@std@@QAE@XZ 004067b0 f i MessageHistory.obj
 0001:000057d0       ??1?$_String_val@U?$_Simple_types@D@std@@@std@@QAE@XZ 004067d0 f i MessageHistory.obj
 0001:000057f0       ??1?$basic_string@DU?$char_traits@D@std@@V?$allocator@D@2@@std@@QAE@XZ 004067f0 f i MessageHistory.obj
 0001:00005840       ?_Orphan_all@_Container_base0@std@@QAEXXZ 00406840 f i MessageHistory.obj
 0001:00005840       ??1_Bxty@?$_String_val@U?$_Simple_types@D@std@@@std@@QAE@XZ 00406840 f i MessageHistory.obj
 0001:00005850       ??2@YAPAXIPAX@Z            00406850 f i MessageHistory.obj
 0001:00005860       ??8?$_List_const_iterator@V?$_List_val@U?$_List_simple_types@V?$basic_string@DU?$char_traits@D@std@@V?$allocator@D@2@@std@@@std@@@std@@@std@@QBE_NABV01@@Z 00406860 f i MessageHistory.obj
 0001:00005890       ??9?$_List_const_iterator@V?$_List_val@U?$_List_simple_types@V?$basic_string@DU?$char_traits@D@std@@V?$allocator@D@2@@std@@@std@@@std@@@std@@QBE_NABV01@@Z 00406890 f i MessageHistory.obj
 0001:000058d0       ??D?$_List_const_iterator@V?$_List_val@U?$_List_simple_types@V?$basic_string@DU?$char_traits@D@std@@V?$allocator@D@2@@std@@@std@@@std@@@std@@QBEABV?$basic_string@DU?$char_traits@D@std@@V?$allocator@D@2@@1@XZ 004068d0 f i MessageHistory.obj
 0001:000058f0       ??E?$_List_const_iterator@V?$_List_val@U?$_List_simple_types@V?$basic_string@DU?$char_traits@D@std@@V?$allocator@D@2@@std@@@std@@@std@@@std@@QAE?AV01@H@Z 004068f0 f i MessageHistory.obj
 0001:00005920       ??E?$_List_const_iterator@V?$_List_val@U?$_List_simple_types@V?$basic_string@DU?$char_traits@D@std@@V?$allocator@D@2@@std@@@std@@@std@@@std@@QAEAAV01@XZ 00406920 f i MessageHistory.obj
 0001:00005940       ??F?$_List_const_iterator@V?$_List_val@U?$_List_simple_types@V?$basic_string@DU?$char_traits@D@std@@V?$allocator@D@2@@std@@@std@@@std@@@std@@QAEAAV01@XZ 00406940 f i MessageHistory.obj
 0001:00005970       ??R<lambda_9366063389c5f42a00a5088cf24e69de>@@QBEXQADIQBD@Z 00406970 f i MessageHistory.obj
 0001:000059b0       ??_G?$basic_string@DU?$char_traits@D@std@@V?$allocator@D@2@@std@@QAEPAXI@Z 004069b0 f i MessageHistory.obj
 0001:000059e0       ?_Adjust_manually_vector_aligned@std@@YAXAAPAXAAI@Z 004069e0 f i MessageHistory.obj
 0001:00005a50       ?_Adopt@_Iterator_base0@std@@QAEXPBX@Z 00406a50 f i MessageHistory.obj
 0001:00005a60       ?_Allocate@_Default_allocate_traits@std@@SAPAXI@Z 00406a60 f i MessageHistory.obj
 0001:00005a80       ?_Assign_rv_contents_with_alloc_always_equal@?$basic_string@DU?$char_traits@D@std@@V?$allocator@D@2@@std@@QAEX$$QAV12@U?$integral_constant@_N$00@2@@Z 00406a80 f i MessageHistory.obj
 0001:00005b10       ?_Buynode0@?$_List_alloc@U?$_List_base_types@V?$basic_string@DU?$char_traits@D@std@@V?$allocator@D@2@@std@@V?$allocator@V?$basic_string@DU?$char_traits@D@std@@V?$allocator@D@2@@std@@@2@@std@@@std@@QAEPAU?$_List_node@V?$basic_string@DU?$char_traits@D@std@@V?$allocator@D@2@@std@@PAX@2@PAU32@0@Z 00406b10 f i MessageHistory.obj
 0001:00005c00       ?_Calculate_growth@?$basic_string@DU?$char_traits@D@std@@V?$allocator@D@2@@std@@QBEII@Z 00406c00 f i MessageHistory.obj
 0001:00005c80       ?_Freenode@?$_List_buy@V?$basic_string@DU?$char_traits@D@std@@V?$allocator@D@2@@std@@V?$allocator@V?$basic_string@DU?$char_traits@D@std@@V?$allocator@D@2@@std@@@2@@std@@QAEXPAU?$_List_node@V?$basic_string@DU?$char_traits@D@std@@V?$allocator@D@2@@std@@PAX@2@@Z 00406c80 f i MessageHistory.obj
 0001:00005cd0       ?_Get_data@?$_List_alloc@U?$_List_base_types@V?$basic_string@DU?$char_traits@D@std@@V?$allocator@D@2@@std@@V?$allocator@V?$basic_string@DU?$char_traits@D@std@@V?$allocator@D@2@@std@@@2@@std@@@std@@QAEAAV?$_List_val@U?$_List_simple_types@V?$basic_string@DU?$char_traits@D@std@@V?$allocator@D@2@@std@@@std@@@2@XZ 00406cd0 f i MessageHistory.obj
 0001:00005cd0       ?_Getal@?$_List_alloc@U?$_List_base_types@V?$basic_string@DU?$char_traits@D@std@@V?$allocator@D@2@@std@@V?$allocator@V?$basic_string@DU?$char_traits@D@std@@V?$allocator@D@2@@std@@@2@@std@@@std@@QBEABV?$allocator@U?$_List_node@V?$basic_string@DU?$char_traits@D@std@@V?$allocator@D@2@@std@@PAX@std@@@2@XZ 00406cd0 f i MessageHistory.obj
 0001:00005cd0       ?_Get_data@?$_String_alloc@U?$_String_base_types@DV?$allocator@D@std@@@std@@@std@@QAEAAV?$_String_val@U?$_Simple_types@D@std@@@2@XZ 00406cd0 f i MessageHistory.obj
 0001:00005cd0       ?_Getal@?$_String_alloc@U?$_String_base_types@DV?$allocator@D@std@@@std@@@std@@QBEABV?$allocator@D@2@XZ 00406cd0 f i MessageHistory.obj
 0001:00005cd0       ?_Get_data@?$_List_alloc@U?$_List_base_types@V?$basic_string@DU?$char_traits@D@std@@V?$allocator@D@2@@std@@V?$allocator@V?$basic_string@DU?$char_traits@D@std@@V?$allocator@D@2@@std@@@2@@std@@@std@@QBEABV?$_List_val@U?$_List_simple_types@V?$basic_string@DU?$char_traits@D@std@@V?$allocator@D@2@@std@@@std@@@2@XZ 00406cd0 f i MessageHistory.obj
 0001:00005cd0       ?_Get_data@?$_String_alloc@U?$_String_base_types@DV?$allocator@D@std@@@std@@@std@@QBEABV?$_String_val@U?$_Simple_types@D@std@@@2@XZ 00406cd0 f i MessageHistory.obj
 0001:00005cd0       ?_Getal@?$_String_alloc@U?$_String_base_types@DV?$allocator@D@std@@@std@@@std@@QAEAAV?$allocator@D@2@XZ 00406cd0 f i MessageHistory.obj
 0001:00005cd0       ?_Getal@?$_List_alloc@U?$_List_base_types@V?$basic_string@DU?$char_traits@D@std@@V?$allocator@D@2@@std@@V?$allocator@V?$basic_string@DU?$char_traits@D@std@@V?$allocator@D@2@@std@@@2@@std@@@std@@QAEAAV?$allocator@U?$_List_node@V?$basic_string@DU?$char_traits@D@std@@V?$allocator@D@2@@std@@PAX@std@@@2@XZ 00406cd0 f i MessageHistory.obj
 0001:00005cf0       ?_Incsize@?$list@V?$basic_string@DU?$char_traits@D@std@@V?$allocator@D@2@@std@@V?$allocator@V?$basic_string@DU?$char_traits@D@std@@V?$allocator@D@2@@std@@@2@@std@@QAEXI@Z 00406cf0 f i MessageHistory.obj
 0001:00005d40       ?_Large_string_engaged@?$_String_val@U?$_Simple_types@D@std@@@std@@QBE_NXZ 00406d40 f i MessageHistory.obj
 0001:00005d70       ?_Make_iter@?$list@V?$basic_string@DU?$char_traits@D@std@@V?$allocator@D@2@@std@@V?$allocator@V?$basic_string@DU?$char_traits@D@std@@V?$allocator@D@2@@std@@@2@@std@@QBE?AV?$_List_iterator@V?$_List_val@U?$_List_simple_types@V?$basic_string@DU?$char_traits@D@std@@V?$allocator@D@2@@std@@@std@@@std@@@2@V?$_List_const_iterator@V?$_List_val@U?$_List_simple_types@V?$basic_string@DU?$char_traits@D@std@@V?$allocator@D@2@@std@@@std@@@std@@@2@@Z 00406d70 f i MessageHistory.obj
 0001:00005dd0       ?_Myhead@?$_List_alloc@U?$_List_base_types@V?$basic_string@DU?$char_traits@D@std@@V?$allocator@D@2@@std@@V?$allocator@V?$basic_string@DU?$char_traits@D@std@@V?$allocator@D@2@@std@@@2@@std@@@std@@QAEAAPAU?$_List_node@V?$basic_string@DU?$char_traits@D@std@@V?$allocator@D@2@@std@@PAX@2@XZ 00406dd0 f i MessageHistory.obj
 0001:00005df0       ?_Myptr@?$_String_val@U?$_Simple_types@D@std@@@std@@QAEPADXZ 00406df0 f i MessageHistory.obj
 0001:00005df0       ?_Myptr@?$_String_val@U?$_Simple_types@D@std@@@std@@QBEPBDXZ 00406df0 f i MessageHistory.obj
 0001:00005e30       ?_Mysize@?$_List_alloc@U?$_List_base_types@V?$basic_string@DU?$char_traits@D@std@@V?$allocator@D@2@@std@@V?$allocator@V?$basic_string@DU?$char_traits@D@std@@V?$allocator@D@2@@std@@@2@@std@@@std@@QBEABIXZ 00406e30 f i MessageHistory.obj
 0001:00005e30       ?_Mysize@?$_List_alloc@U?$_List_base_types@V?$basic_string@DU?$char_traits@D@std@@V?$allocator@D@2@@std@@V?$allocator@V?$basic_string@DU?$char_traits@D@std@@V?$allocator@D@2@@std@@@2@@std@@@std@@QAEAAIXZ 00406e30 f i MessageHistory.obj
 0001:00005e50       ?_Orphan_all@?$_String_alloc@U?$_String_base_types@DV?$allocator@D@std@@@std@@@std@@QAEXXZ 00406e50 f i MessageHistory.obj
 0001:00005e70       ?_Tidy_deallocate@?$basic_string@DU?$char_traits@D@std@@V?$allocator@D@2@@std@@QAEXXZ 00406e70 f i MessageHistory.obj
 0001:00005f20       ?_Tidy_init@?$basic_string@DU?$char_traits@D@std@@V?$allocator@D@2@@std@@QAEXXZ 00406f20 f i MessageHistory.obj
 0001:00005f70       ?_Unchecked_end@?$list@V?$basic_string@DU?$char_traits@D@std@@V?$allocator@D@2@@std@@V?$allocator@V?$basic_string@DU?$char_traits@D@std@@V?$allocator@D@2@@std@@@2@@std@@QAE?AV?$_List_unchecked_iterator@V?$_List_val@U?$_List_simple_types@V?$basic_string@DU?$char_traits@D@std@@V?$allocator@D@2@@std@@@std@@@std@@@2@XZ 00406f70 f i MessageHistory.obj
 0001:00005fa0       ?_Unlinknode@?$list@V?$basic_string@DU?$char_traits@D@std@@V?$allocator@D@2@@std@@V?$allocator@V?$basic_string@DU?$char_traits@D@std@@V?$allocator@D@2@@std@@@2@@std@@QAEPAU?$_List_node@V?$basic_string@DU?$char_traits@D@std@@V?$allocator@D@2@@std@@PAX@2@V?$_List_const_iterator@V?$_List_val@U?$_List_simple_types@V?$basic_string@DU?$char_traits@D@std@@V?$allocator@D@2@@std@@@std@@@std@@@2@@Z 00406fa0 f i MessageHistory.obj
 0001:00005ff0       ?_Xlen@?$basic_string@DU?$char_traits@D@std@@V?$allocator@D@2@@std@@SAXXZ 00406ff0 f i MessageHistory.obj
 0001:00006000       ?allocate@?$allocator@D@std@@QAEPADI@Z 00407000 f i MessageHistory.obj
 0001:00006030       ?allocate@?$allocator@U?$_List_node@V?$basic_string@DU?$char_traits@D@std@@V?$allocator@D@2@@std@@PAX@std@@@std@@QAEPAU?$_List_node@V?$basic_string@DU?$char_traits@D@std@@V?$allocator@D@2@@std@@PAX@2@I@Z 00407030 f i MessageHistory.obj
 0001:00006060       ?assign@?$basic_string@DU?$char_traits@D@std@@V?$allocator@D@2@@std@@QAEAAV12@QBD@Z 00407060 f i MessageHistory.obj
 0001:00006090       ?assign@?$basic_string@DU?$char_traits@D@std@@V?$allocator@D@2@@std@@QAEAAV12@QBDI@Z 00407090 f i MessageHistory.obj
 0001:00006120       ?assign@?$char_traits@D@std@@SAXAADABD@Z 00407120 f i MessageHistory.obj
 0001:00006130       ?begin@?$list@V?$basic_string@DU?$char_traits@D@std@@V?$allocator@D@2@@std@@V?$allocator@V?$basic_string@DU?$char_traits@D@std@@V?$allocator@D@2@@std@@@2@@std@@QAE?AV?$_List_iterator@V?$_List_val@U?$_List_simple_types@V?$basic_string@DU?$char_traits@D@std@@V?$allocator@D@2@@std@@@std@@@std@@@2@XZ 00407130 f i MessageHistory.obj
 0001:000061a0       ?c_str@?$basic_string@DU?$char_traits@D@std@@V?$allocator@D@2@@std@@QBEPBDXZ 004071a0 f i MessageHistory.obj
 0001:000061f0       ?clear@?$list@V?$basic_string@DU?$char_traits@D@std@@V?$allocator@D@2@@std@@V?$allocator@V?$basic_string@DU?$char_traits@D@std@@V?$allocator@D@2@@std@@@2@@std@@QAEXXZ 004071f0 f i MessageHistory.obj
 0001:000062b0       ?copy@?$char_traits@D@std@@SAPADQADQBDI@Z 004072b0 f i MessageHistory.obj
 0001:000062d0       ?deallocate@?$_Default_allocator_traits@V?$allocator@U?$_List_node@V?$basic_string@DU?$char_traits@D@std@@V?$allocator@D@2@@std@@PAX@std@@@std@@@std@@SAXAAV?$allocator@U?$_List_node@V?$basic_string@DU?$char_traits@D@std@@V?$allocator@D@2@@std@@PAX@std@@@2@QAU?$_List_node@V?$basic_string@DU?$char_traits@D@std@@V?$allocator@D@2@@std@@PAX@2@I@Z 004072d0 f i MessageHistory.obj
 0001:000062f0       ?deallocate@?$allocator@D@std@@QAEXQADI@Z 004072f0 f i MessageHistory.obj
 0001:00006310       ?deallocate@?$allocator@U?$_List_node@V?$basic_string@DU?$char_traits@D@std@@V?$allocator@D@2@@std@@PAX@std@@@std@@QAEXQAU?$_List_node@V?$basic_string@DU?$char_traits@D@std@@V?$allocator@D@2@@std@@PAX@2@I@Z 00407310 f i MessageHistory.obj
 0001:00006330       ?empty@?$list@V?$basic_string@DU?$char_traits@D@std@@V?$allocator@D@2@@std@@V?$allocator@V?$basic_string@DU?$char_traits@D@std@@V?$allocator@D@2@@std@@@2@@std@@QBE_NXZ 00407330 f i MessageHistory.obj
 0001:00006360       ?end@?$list@V?$basic_string@DU?$char_traits@D@std@@V?$allocator@D@2@@std@@V?$allocator@V?$basic_string@DU?$char_traits@D@std@@V?$allocator@D@2@@std@@@2@@std@@QAE?AV?$_List_iterator@V?$_List_val@U?$_List_simple_types@V?$basic_string@DU?$char_traits@D@std@@V?$allocator@D@2@@std@@@std@@@std@@@2@XZ 00407360 f i MessageHistory.obj
 0001:000063c0       ?erase@?$list@V?$basic_string@DU?$char_traits@D@std@@V?$allocator@D@2@@std@@V?$allocator@V?$basic_string@DU?$char_traits@D@std@@V?$allocator@D@2@@std@@@2@@std@@QAE?AV?$_List_iterator@V?$_List_val@U?$_List_simple_types@V?$basic_string@DU?$char_traits@D@std@@V?$allocator@D@2@@std@@@std@@@std@@@2@V?$_List_const_iterator@V?$_List_val@U?$_List_simple_types@V?$basic_string@DU?$char_traits@D@std@@V?$allocator@D@2@@std@@@std@@@std@@@2@@Z 004073c0 f i MessageHistory.obj
 0001:00006410       ?length@?$char_traits@D@std@@SAIQBD@Z 00407410 f i MessageHistory.obj
 0001:00006430       ?max@?$numeric_limits@H@std@@SAHXZ 00407430 f i MessageHistory.obj
 0001:00006440       ?max_size@?$_Default_allocator_traits@V?$allocator@D@std@@@std@@SAIABV?$allocator@D@2@@Z 00407440 f i MessageHistory.obj
 0001:00006450       ?max_size@?$_Default_allocator_traits@V?$allocator@U?$_List_node@V?$basic_string@DU?$char_traits@D@std@@V?$allocator@D@2@@std@@PAX@std@@@std@@@std@@SAIABV?$allocator@U?$_List_node@V?$basic_string@DU?$char_traits@D@std@@V?$allocator@D@2@@std@@PAX@std@@@2@@Z 00407450 f i MessageHistory.obj
 0001:00006460       ?max_size@?$basic_string@DU?$char_traits@D@std@@V?$allocator@D@2@@std@@QBEIXZ 00407460 f i MessageHistory.obj
 0001:000064c0       ?max_size@?$list@V?$basic_string@DU?$char_traits@D@std@@V?$allocator@D@2@@std@@V?$allocator@V?$basic_string@DU?$char_traits@D@std@@V?$allocator@D@2@@std@@@2@@std@@QBEIXZ 004074c0 f i MessageHistory.obj
 0001:000064e0       ?move@?$char_traits@D@std@@SAPADQADQBDI@Z 004074e0 f i MessageHistory.obj
 0001:00006500       ?pop_front@?$list@V?$basic_string@DU?$char_traits@D@std@@V?$allocator@D@2@@std@@V?$allocator@V?$basic_string@DU?$char_traits@D@std@@V?$allocator@D@2@@std@@@2@@std@@QAEXXZ 00407500 f i MessageHistory.obj
 0001:00006530       ?push_back@?$list@V?$basic_string@DU?$char_traits@D@std@@V?$allocator@D@2@@std@@V?$allocator@V?$basic_string@DU?$char_traits@D@std@@V?$allocator@D@2@@std@@@2@@std@@QAEX$$QAV?$basic_string@DU?$char_traits@D@std@@V?$allocator@D@2@@2@@Z 00407530 f i MessageHistory.obj
 0001:00006570       ?size@?$list@V?$basic_string@DU?$char_traits@D@std@@V?$allocator@D@2@@std@@V?$allocator@V?$basic_string@DU?$char_traits@D@std@@V?$allocator@D@2@@std@@@2@@std@@QBEIXZ 00407570 f i MessageHistory.obj
 0001:000065d0       _WinMain@16                004075d0 f   jaccessinspector.obj
 0001:00006720       ?TimerProc@@YGXPAUHWND__@@IIK@Z 00407720 f   jaccessinspector.obj
 0001:00006760       ?KeyboardProc@@YGJHIJ@Z    00407760 f   jaccessinspector.obj
 0001:00006800       ?MouseProc@@YGJHIJ@Z       00407800 f   jaccessinspector.obj
 0001:00006860       ?InitWindow@@YAHPAX@Z      00407860 f   jaccessinspector.obj
 0001:00006900       ?jaccessinspectorDialogProc@@YGHPAUHWND__@@IIJ@Z 00407900 f   jaccessinspector.obj
 0001:00008370       ?HandleJavaShutdown@@YAXJ@Z 00409370 f   jaccessinspector.obj
 0001:000083f0       ?HandleJavaFocusGained@@YAXJ_J0@Z 004093f0 f   jaccessinspector.obj
 0001:00008480       ?HandleJavaFocusLost@@YAXJ_J0@Z 00409480 f   jaccessinspector.obj
 0001:00008510       ?HandleJavaCaretUpdate@@YAXJ_J0@Z 00409510 f   jaccessinspector.obj
 0001:00008560       ?HandleMouseClicked@@YAXJ_J0@Z 00409560 f   jaccessinspector.obj
 0001:000085b0       ?HandleMouseEntered@@YAXJ_J0@Z 004095b0 f   jaccessinspector.obj
 0001:00008600       ?HandleMouseExited@@YAXJ_J0@Z 00409600 f   jaccessinspector.obj
 0001:00008650       ?HandleMousePressed@@YAXJ_J0@Z 00409650 f   jaccessinspector.obj
 0001:000086a0       ?HandleMouseReleased@@YAXJ_J0@Z 004096a0 f   jaccessinspector.obj
 0001:000086f0       ?HandleMenuCanceled@@YAXJ_J0@Z 004096f0 f   jaccessinspector.obj
 0001:00008740       ?HandleMenuDeselected@@YAXJ_J0@Z 00409740 f   jaccessinspector.obj
 0001:00008790       ?HandleMenuSelected@@YAXJ_J0@Z 00409790 f   jaccessinspector.obj
 0001:000087e0       ?HandlePopupMenuCanceled@@YAXJ_J0@Z 004097e0 f   jaccessinspector.obj
 0001:00008830       ?HandlePopupMenuWillBecomeInvisible@@YAXJ_J0@Z 00409830 f   jaccessinspector.obj
 0001:00008880       ?HandlePopupMenuWillBecomeVisible@@YAXJ_J0@Z 00409880 f   jaccessinspector.obj
 0001:000088d0       ?HandlePropertyNameChange@@YAXJ_J0PAG1@Z 004098d0 f   jaccessinspector.obj
 0001:00008960       ?HandlePropertyDescriptionChange@@YAXJ_J0PAG1@Z 00409960 f   jaccessinspector.obj
 0001:000089f0       ?HandlePropertyStateChange@@YAXJ_J0PAG1@Z 004099f0 f   jaccessinspector.obj
 0001:00008a80       ?HandlePropertyValueChange@@YAXJ_J0PAG1@Z 00409a80 f   jaccessinspector.obj
 0001:00008b10       ?HandlePropertySelectionChange@@YAXJ_J0@Z 00409b10 f   jaccessinspector.obj
 0001:00008b60       ?HandlePropertyTextChange@@YAXJ_J0@Z 00409b60 f   jaccessinspector.obj
 0001:00008bb0       ?HandlePropertyCaretChange@@YAXJ_J0HH@Z 00409bb0 f   jaccessinspector.obj
 0001:00008c40       ?HandlePropertyVisibleDataChange@@YAXJ_J0@Z 00409c40 f   jaccessinspector.obj
 0001:00008c90       ?HandlePropertyTableModelChange@@YAXJ_J0PAG1@Z 00409c90 f   jaccessinspector.obj
 0001:00008d20       ?SaveActiveEventOptionsToRegistry@@YAHXZ 00409d20 f   jaccessinspector.obj
 0001:00009230       ?ReadActiveEventOptionsFromRegistry@@YAHXZ 0040a230 f   jaccessinspector.obj
 0001:00009c30       ?ApplyEventOptions@@YAXPAUHWND__@@@Z 0040ac30 f   jaccessinspector.obj
 0001:0000a350       ?EnableDlgItem@@YAHPAUHWND__@@HH@Z 0040b350 f   jaccessinspector.obj
 0001:0000a390       ?EnableMessageNavButtons@@YAXXZ 0040b390 f   jaccessinspector.obj
 0001:0000a610       ?AddToMessageHistory@@YGXPBD@Z 0040b610 f   jaccessinspector.obj
 0001:0000a630       ?UpdateMessageNumber@@YAHXZ 0040b630 f   jaccessinspector.obj
 0001:0000a6e0       ?GoToMessageDialogProc@@YGHPAUHWND__@@IIJ@Z 0040b6e0 f   jaccessinspector.obj
 0001:0000a960       ?InitGoToMessageDialogBox@@YAHPAX@Z 0040b960 f   jaccessinspector.obj
 0001:0000a9b0       ?ShouldCheckMonitorTheSameEventsAsJAWS@@YAHXZ 0040b9b0 f   jaccessinspector.obj
 0001:0000aae0       ?MaybeCheckMonitorTheSameEventsAsJAWS@@YAXPAUHMENU__@@@Z 0040bae0 f   jaccessinspector.obj
 0001:0000ab20       ?ShouldCheckMonitorAllEvents@@YAHXZ 0040bb20 f   jaccessinspector.obj
 0001:0000ac50       ?MaybeCheckMonitorAllEvents@@YAXPAUHMENU__@@@Z 0040bc50 f   jaccessinspector.obj
 0001:0000ac90       ?displayAccessibleInfo@@YAXJ_JHH@Z 0040bc90 f   jaccessinspector.obj
 0001:0000ad00       ?displayJavaEvent@@YAXJ_JPAD@Z 0040bd00 f   jaccessinspector.obj
 0001:0000adc0       ?displayAccessiblePropertyChange@@YAXJ_JPAD@Z 0040bdc0 f   jaccessinspector.obj
 0001:0000ae80       ?echoMouseObject@@YAXXZ    0040be80 f   jaccessinspector.obj
 0001:0000af40       ?echoMouseHWNDObject@@YAXXZ 0040bf40 f   jaccessinspector.obj
 0001:0000afb0       ?displayFocusedObject@@YAXXZ 0040bfb0 f   jaccessinspector.obj
 0001:0000b040       ?HandlePropertyChildChange@@YAXJ_J000@Z 0040c040 f   jaccessinspector.obj
 0001:0000b210       ?HandlePropertyActiveDescendentChange@@YAXJ_J000@Z 0040c210 f   jaccessinspector.obj
 0001:0000b2c0       ?exitjaccessinspector@@YAXPAUHWND__@@@Z 0040c2c0 f   jaccessinspector.obj
 0001:0000b2e0       ?reinstallEventListeners@@YAXXZ 0040c2e0 f   jaccessinspector.obj
 0001:0000b530       ??$?0$$V@?$_Compressed_pair@V?$allocator@U?$_List_node@V?$basic_string@DU?$char_traits@D@std@@V?$allocator@D@2@@std@@PAX@std@@@std@@V?$_List_val@U?$_List_simple_types@V?$basic_string@DU?$char_traits@D@std@@V?$allocator@D@2@@std@@@std@@@2@$00@std@@QAE@U_Zero_then_variadic_args_t@1@@Z 0040c530 f i jaccessinspector.obj
 0001:0000b550       ??0?$_List_alloc@U?$_List_base_types@V?$basic_string@DU?$char_traits@D@std@@V?$allocator@D@2@@std@@V?$allocator@V?$basic_string@DU?$char_traits@D@std@@V?$allocator@D@2@@std@@@2@@std@@@std@@QAE@XZ 0040c550 f i jaccessinspector.obj
 0001:0000b590       ??0?$_List_buy@V?$basic_string@DU?$char_traits@D@std@@V?$allocator@D@2@@std@@V?$allocator@V?$basic_string@DU?$char_traits@D@std@@V?$allocator@D@2@@std@@@2@@std@@QAE@XZ 0040c590 f i jaccessinspector.obj
 0001:0000b5b0       ??0?$_List_const_iterator@V?$_List_val@U?$_List_simple_types@V?$basic_string@DU?$char_traits@D@std@@V?$allocator@D@2@@std@@@std@@@std@@@std@@QAE@XZ 0040c5b0 f i jaccessinspector.obj
 0001:0000b5d0       ??0?$_List_unchecked_const_iterator@V?$_List_val@U?$_List_simple_types@V?$basic_string@DU?$char_traits@D@std@@V?$allocator@D@2@@std@@@std@@@std@@U_Iterator_base0@2@@std@@QAE@XZ 0040c5d0 f i jaccessinspector.obj
 0001:0000b5f0       ??0?$_List_val@U?$_List_simple_types@V?$basic_string@DU?$char_traits@D@std@@V?$allocator@D@2@@std@@@std@@@std@@QAE@XZ 0040c5f0 f i jaccessinspector.obj
 0001:0000b620       ??0?$list@V?$basic_string@DU?$char_traits@D@std@@V?$allocator@D@2@@std@@V?$allocator@V?$basic_string@DU?$char_traits@D@std@@V?$allocator@D@2@@std@@@2@@std@@QAE@XZ 0040c620 f i jaccessinspector.obj
 0001:0000b640       ??0MessageHistory@@QAE@XZ  0040c640 f i jaccessinspector.obj
 0001:0000b6a0       ??1?$_List_alloc@U?$_List_base_types@V?$basic_string@DU?$char_traits@D@std@@V?$allocator@D@2@@std@@V?$allocator@V?$basic_string@DU?$char_traits@D@std@@V?$allocator@D@2@@std@@@2@@std@@@std@@QAE@XZ 0040c6a0 f i jaccessinspector.obj
 0001:0000b6f0       ??1?$_List_buy@V?$basic_string@DU?$char_traits@D@std@@V?$allocator@D@2@@std@@V?$allocator@V?$basic_string@DU?$char_traits@D@std@@V?$allocator@D@2@@std@@@2@@std@@QAE@XZ 0040c6f0 f i jaccessinspector.obj
 0001:0000b710       ??1?$list@V?$basic_string@DU?$char_traits@D@std@@V?$allocator@D@2@@std@@V?$allocator@V?$basic_string@DU?$char_traits@D@std@@V?$allocator@D@2@@std@@@2@@std@@QAE@XZ 0040c710 f i jaccessinspector.obj
 0001:0000b760       ??1MessageHistory@@QAE@XZ  0040c760 f i jaccessinspector.obj
 0001:0000b780       ?_Buyheadnode@?$_List_alloc@U?$_List_base_types@V?$basic_string@DU?$char_traits@D@std@@V?$allocator@D@2@@std@@V?$allocator@V?$basic_string@DU?$char_traits@D@std@@V?$allocator@D@2@@std@@@2@@std@@@std@@QAEPAU?$_List_node@V?$basic_string@DU?$char_traits@D@std@@V?$allocator@D@2@@std@@PAX@2@XZ 0040c780 f i jaccessinspector.obj
 0001:0000b7a0       ?_Freeheadnode@?$_List_alloc@U?$_List_base_types@V?$basic_string@DU?$char_traits@D@std@@V?$allocator@D@2@@std@@V?$allocator@V?$basic_string@DU?$char_traits@D@std@@V?$allocator@D@2@@std@@@2@@std@@@std@@QAEXPAU?$_List_node@V?$basic_string@DU?$char_traits@D@std@@V?$allocator@D@2@@std@@PAX@2@@Z 0040c7a0 f i jaccessinspector.obj
 0001:0000b7d0       ?_Tidy@?$list@V?$basic_string@DU?$char_traits@D@std@@V?$allocator@D@2@@std@@V?$allocator@V?$basic_string@DU?$char_traits@D@std@@V?$allocator@D@2@@std@@@2@@std@@QAEXXZ 0040c7d0 f i jaccessinspector.obj
 0001:0000b7f0       __snprintf                 0040c7f0 f i jaccessinspector.obj
 0001:0000b830       __vsnprintf                0040c830 f i jaccessinspector.obj
 0001:0000b84f       ??_U@YAPAXI@Z              0040c84f f   MSVCRT:new_array.obj
 0001:0000b858       ??_V@YAXPAX@Z              0040c858 f   MSVCRT:delete_array.obj
 0001:0000b85d       ___raise_securityfailure   0040c85d f   MSVCRT:gs_report.obj
 0001:0000b885       ___report_gsfailure        0040c885 f   MSVCRT:gs_report.obj
 0001:0000b97e       ___report_rangecheckfailure 0040c97e f   MSVCRT:gs_report.obj
 0001:0000b98a       ___report_securityfailure  0040c98a f   MSVCRT:gs_report.obj
 0001:0000ba60       __aulldiv                  0040ca60 f   MSVCRT:ulldiv.obj
 0001:0000bac8       @__security_check_cookie@4 0040cac8 f   MSVCRT:secchk.obj
 0001:0000bae0       __alloca_probe             0040cae0 f   MSVCRT:chkstk.obj
 0001:0000bae0       __chkstk                   0040cae0 f   MSVCRT:chkstk.obj
 0001:0000bb0d       ??2@YAPAXI@Z               0040cb0d f   MSVCRT:new_scalar.obj
 0001:0000bb3d       ??3@YAXPAXI@Z              0040cb3d f   MSVCRT:delete_scalar_size.obj
 0001:0000bb8f       ___scrt_acquire_startup_lock 0040cb8f f   MSVCRT:utility.obj
 0001:0000bbc1       ___scrt_initialize_crt     0040cbc1 f   MSVCRT:utility.obj
 0001:0000bbfa       ___scrt_initialize_onexit_tables 0040cbfa f   MSVCRT:utility.obj
 0001:0000bc9f       ___scrt_is_nonwritable_in_current_image 0040cc9f f   MSVCRT:utility.obj
 0001:0000bd33       ___scrt_release_startup_lock 0040cd33 f   MSVCRT:utility.obj
 0001:0000bd50       ___scrt_uninitialize_crt   0040cd50 f   MSVCRT:utility.obj
 0001:0000bd78       __onexit                   0040cd78 f   MSVCRT:utility.obj
 0001:0000bdb3       _atexit                    0040cdb3 f   MSVCRT:utility.obj
 0001:0000bdef       ??$__crt_fast_encode_pointer@P6GHPAU_RTL_CONDITION_VARIABLE@@PAU_RTL_CRITICAL_SECTION@@K@Z@@YAP6GHPAU_RTL_CONDITION_VARIABLE@@PAU_RTL_CRITICAL_SECTION@@K@ZQ6GH01K@Z@Z 0040cdef f i MSVCRT:thread_safe_statics.obj
 0001:0000bdef       ??$__crt_fast_encode_pointer@P6GXPAU_RTL_CONDITION_VARIABLE@@@Z@@YAP6GXPAU_RTL_CONDITION_VARIABLE@@@ZQ6GX0@Z@Z 0040cdef f i MSVCRT:thread_safe_statics.obj
 0001:0000bf17       __Init_thread_footer       0040cf17 f   MSVCRT:thread_safe_statics.obj
 0001:0000bf61       __Init_thread_header       0040cf61 f   MSVCRT:thread_safe_statics.obj
 0001:0000bfb3       __Init_thread_notify       0040cfb3 f   MSVCRT:thread_safe_statics.obj
 0001:0000bff5       __Init_thread_wait         0040cff5 f   MSVCRT:thread_safe_statics.obj
 0001:0000c296       _WinMainCRTStartup         0040d296 f   MSVCRT:exe_winmain.obj
 0001:0000c2a0       ??3@YAXPAX@Z               0040d2a0 f   MSVCRT:delete_scalar.obj
 0001:0000c2a5       ??0bad_alloc@std@@QAE@ABV01@@Z 0040d2a5 f i MSVCRT:throw_bad_alloc.obj
 0001:0000c2c0       ??0bad_alloc@std@@QAE@XZ   0040d2c0 f i MSVCRT:throw_bad_alloc.obj
 0001:0000c2d8       ??0bad_array_new_length@std@@QAE@ABV01@@Z 0040d2d8 f i MSVCRT:throw_bad_alloc.obj
 0001:0000c2f3       ??0bad_array_new_length@std@@QAE@XZ 0040d2f3 f i MSVCRT:throw_bad_alloc.obj
 0001:0000c30b       ??0exception@std@@QAE@ABV01@@Z 0040d30b f i MSVCRT:throw_bad_alloc.obj
 0001:0000c337       ??1bad_alloc@std@@UAE@XZ   0040d337 f i MSVCRT:throw_bad_alloc.obj
 0001:0000c337       ??1bad_array_new_length@std@@UAE@XZ 0040d337 f i MSVCRT:throw_bad_alloc.obj
 0001:0000c348       ??_Ebad_array_new_length@std@@UAEPAXI@Z 0040d348 f i MSVCRT:throw_bad_alloc.obj
 0001:0000c348       ??_Gbad_alloc@std@@UAEPAXI@Z 0040d348 f i MSVCRT:throw_bad_alloc.obj
 0001:0000c348       ??_Ebad_alloc@std@@UAEPAXI@Z 0040d348 f i MSVCRT:throw_bad_alloc.obj
 0001:0000c348       ??_Gexception@std@@UAEPAXI@Z 0040d348 f i MSVCRT:throw_bad_alloc.obj
 0001:0000c348       ??_Gbad_array_new_length@std@@UAEPAXI@Z 0040d348 f i MSVCRT:throw_bad_alloc.obj
 0001:0000c348       ??_Eexception@std@@UAEPAXI@Z 0040d348 f i MSVCRT:throw_bad_alloc.obj
 0001:0000c375       ?__scrt_throw_std_bad_alloc@@YAXXZ 0040d375 f   MSVCRT:throw_bad_alloc.obj
 0001:0000c392       ?__scrt_throw_std_bad_array_new_length@@YAXXZ 0040d392 f   MSVCRT:throw_bad_alloc.obj
 0001:0000c3af       ?what@exception@std@@UBEPBDXZ 0040d3af f i MSVCRT:throw_bad_alloc.obj
 0001:0000c3bc       ___isa_available_init      0040d3bc f   MSVCRT:cpu_disp.obj
 0001:0000c553       __get_startup_argv_mode    0040d553 f   MSVCRT:argv_mode.obj
 0001:0000c557       ___scrt_is_ucrt_dll_in_use 0040d557 f   MSVCRT:ucrt_detection.obj
 0001:0000c563       ___scrt_fastfail           0040d563 f   MSVCRT:utility_desktop.obj
 0001:0000c67d       ___scrt_get_show_window_mode 0040d67d f   MSVCRT:utility_desktop.obj
 0001:0000c6ae       ___scrt_initialize_mta     0040d6ae f   MSVCRT:utility_desktop.obj
 0001:0000c6b3       __get_startup_commit_mode  0040d6b3 f   MSVCRT:commit_mode.obj
 0001:0000c6b3       ___scrt_exe_initialize_mta 0040d6b3 f   MSVCRT:utility_desktop.obj
 0001:0000c6b3       ___scrt_initialize_winrt   0040d6b3 f   MSVCRT:utility_desktop.obj
 0001:0000c6b3       __matherr                  0040d6b3 f   MSVCRT:matherr.obj
 0001:0000c6b3       __get_startup_thread_locale_mode 0040d6b3 f   MSVCRT:thread_locale.obj
 0001:0000c6b3       __get_startup_new_mode     0040d6b3 f   MSVCRT:new_mode.obj
 0001:0000c6b3       ___scrt_stub_for_initialize_mta 0040d6b3 f   MSVCRT:utility_desktop.obj
 0001:0000c6b6       ___scrt_is_managed_app     0040d6b6 f   MSVCRT:utility_desktop.obj
 0001:0000c6f9       ___scrt_set_unhandled_exception_filter 0040d6f9 f   MSVCRT:utility_desktop.obj
 0001:0000c705       ___scrt_unhandled_exception_filter@4 0040d705 f   MSVCRT:utility_desktop.obj
 0001:0000c746       __crt_debugger_hook        0040d746 f   MSVCRT:utility_desktop.obj
 0001:0000c750       __SEH_prolog4              0040d750 f   MSVCRT:sehprolg4.obj
 0001:0000c796       __SEH_epilog4              0040d796 f   MSVCRT:sehprolg4.obj
 0001:0000c7ab       __except_handler4          0040d7ab f   MSVCRT:chandler4gs.obj
 0001:0000c7ce       @_guard_check_icall_nop@4  0040d7ce f i MSVCRT:guard_support.obj
 0001:0000c7ce       __initialize_invalid_parameter_handler 0040d7ce f i MSVCRT:invalid_parameter_handler.obj
 0001:0000c7ce       __initialize_denormal_control 0040d7ce f i MSVCRT:denormal_control.obj
 0001:0000c81c       ___security_init_cookie    0040d81c f   MSVCRT:gs_support.obj
 0001:0000c867       __get_startup_file_mode    0040d867 f   MSVCRT:file_mode.obj
 0001:0000c86d       ?__scrt_initialize_type_info@@YAXXZ 0040d86d f   MSVCRT:tncleanup.obj
 0001:0000c879       ___scrt_stub_for_acrt_uninitialize 0040d879 f   MSVCRT:ucrt_stubs.obj
 0001:0000c879       ___acrt_initialize         0040d879 f   MSVCRT:ucrt_stubs.obj
 0001:0000c879       ___acrt_uninitialize       0040d879 f   MSVCRT:ucrt_stubs.obj
 0001:0000c879       ___vcrt_uninitialize       0040d879 f   MSVCRT:ucrt_stubs.obj
 0001:0000c879       ___scrt_stub_for_acrt_initialize 0040d879 f   MSVCRT:ucrt_stubs.obj
 0001:0000c879       __should_initialize_environment 0040d879 f   MSVCRT:env_mode.obj
 0001:0000c879       ___vcrt_initialize         0040d879 f   MSVCRT:ucrt_stubs.obj
 0001:0000c87c       __initialize_default_precision 0040d87c f   MSVCRT:default_precision.obj
 0001:0000c89d       ___local_stdio_scanf_options 0040d89d f i MSVCRT:default_local_stdio_options.obj
 0001:0000c8a3       ___scrt_initialize_default_local_stdio_options 0040d8a3 f   MSVCRT:default_local_stdio_options.obj
 0001:0000c8c0       ___scrt_is_user_matherr_present 0040d8c0 f   MSVCRT:matherr_detection.obj
 0001:0000c8cc       ___scrt_get_dyn_tls_init_callback 0040d8cc f   MSVCRT:dyn_tls_init.obj
 0001:0000c8d2       ___scrt_get_dyn_tls_dtor_callback 0040d8d2 f   MSVCRT:dyn_tls_dtor.obj
 0001:0000c8d8       __RTC_Initialize           0040d8d8 f   MSVCRT:initsect.obj
 0001:0000c904       __RTC_Terminate            0040d904 f   MSVCRT:initsect.obj
 0001:0000c930       ??_Gtype_info@@UAEPAXI@Z   0040d930 f i MSVCRT:std_type_info_static.obj
 0001:0000c930       ??_Etype_info@@UAEPAXI@Z   0040d930 f i MSVCRT:std_type_info_static.obj
 0001:0000c953       ?_Xlength_error@std@@YAXPBD@Z 0040d953 f   msvcprt:MSVCP140.dll
 0001:0000c959       _IsProcessorFeaturePresent@4 0040d959 f   kernel32:KERNEL32.dll
 0001:0000c95f       _memcpy                    0040d95f f   vcruntime:VCRUNTIME140.dll
 0001:0000c965       _memset                    0040d965 f   vcruntime:VCRUNTIME140.dll
 0001:0000c96b       _memmove                   0040d96b f   vcruntime:VCRUNTIME140.dll
 0001:0000c971       __CxxThrowException@8      0040d971 f   vcruntime:VCRUNTIME140.dll
 0001:0000c977       ___CxxFrameHandler3        0040d977 f   vcruntime:VCRUNTIME140.dll
 0001:0000c97d       ___std_exception_copy      0040d97d f   vcruntime:VCRUNTIME140.dll
 0001:0000c983       ___std_exception_destroy   0040d983 f   vcruntime:VCRUNTIME140.dll
 0001:0000c989       __except_handler4_common   0040d989 f   vcruntime:VCRUNTIME140.dll
 0001:0000c98f       _strlen                    0040d98f f   ucrt:api-ms-win-crt-string-l1-1-0.dll
 0001:0000c995       _strcpy                    0040d995 f   ucrt:api-ms-win-crt-string-l1-1-0.dll
 0001:0000c99b       __callnewh                 0040d99b f   ucrt:api-ms-win-crt-heap-l1-1-0.dll
 0001:0000c9a1       _malloc                    0040d9a1 f   ucrt:api-ms-win-crt-heap-l1-1-0.dll
 0001:0000c9a7       __configure_narrow_argv    0040d9a7 f   ucrt:api-ms-win-crt-runtime-l1-1-0.dll
 0001:0000c9ad       __initialize_narrow_environment 0040d9ad f   ucrt:api-ms-win-crt-runtime-l1-1-0.dll
 0001:0000c9b3       __initialize_onexit_table  0040d9b3 f   ucrt:api-ms-win-crt-runtime-l1-1-0.dll
 0001:0000c9b9       __register_onexit_function 0040d9b9 f   ucrt:api-ms-win-crt-runtime-l1-1-0.dll
 0001:0000c9bf       __crt_atexit               0040d9bf f   ucrt:api-ms-win-crt-runtime-l1-1-0.dll
 0001:0000c9c5       __cexit                    0040d9c5 f   ucrt:api-ms-win-crt-runtime-l1-1-0.dll
 0001:0000c9cb       __seh_filter_exe           0040d9cb f   ucrt:api-ms-win-crt-runtime-l1-1-0.dll
 0001:0000c9d1       __set_app_type             0040d9d1 f   ucrt:api-ms-win-crt-runtime-l1-1-0.dll
 0001:0000c9d7       ___setusermatherr          0040d9d7 f   ucrt:api-ms-win-crt-math-l1-1-0.dll
 0001:0000c9dd       __get_narrow_winmain_command_line 0040d9dd f   ucrt:api-ms-win-crt-runtime-l1-1-0.dll
 0001:0000c9e3       __initterm                 0040d9e3 f   ucrt:api-ms-win-crt-runtime-l1-1-0.dll
 0001:0000c9e9       __initterm_e               0040d9e9 f   ucrt:api-ms-win-crt-runtime-l1-1-0.dll
 0001:0000c9ef       _exit                      0040d9ef f   ucrt:api-ms-win-crt-runtime-l1-1-0.dll
 0001:0000c9f5       __exit                     0040d9f5 f   ucrt:api-ms-win-crt-runtime-l1-1-0.dll
 0001:0000c9fb       __set_fmode                0040d9fb f   ucrt:api-ms-win-crt-stdio-l1-1-0.dll
 0001:0000ca01       __c_exit                   0040da01 f   ucrt:api-ms-win-crt-runtime-l1-1-0.dll
 0001:0000ca07       __register_thread_local_exe_atexit_callback 0040da07 f   ucrt:api-ms-win-crt-runtime-l1-1-0.dll
 0001:0000ca0d       __configthreadlocale       0040da0d f   ucrt:api-ms-win-crt-locale-l1-1-0.dll
 0001:0000ca13       __set_new_mode             0040da13 f   ucrt:api-ms-win-crt-heap-l1-1-0.dll
 0001:0000ca19       ___p__commode              0040da19 f   ucrt:api-ms-win-crt-stdio-l1-1-0.dll
 0001:0000ca1f       _free                      0040da1f f   ucrt:api-ms-win-crt-heap-l1-1-0.dll
 0001:0000ca25       _terminate                 0040da25 f   ucrt:api-ms-win-crt-runtime-l1-1-0.dll
 0001:0000ca2b       __controlfp_s              0040da2b f   ucrt:api-ms-win-crt-runtime-l1-1-0.dll
 0002:00000000       __imp__RegCreateKeyExA@36  0040e000     advapi32:ADVAPI32.dll
 0002:00000004       __imp__RegFlushKey@4       0040e004     advapi32:ADVAPI32.dll
 0002:00000008       __imp__RegOpenKeyExA@20    0040e008     advapi32:ADVAPI32.dll
 0002:0000000c       __imp__RegQueryValueExA@24 0040e00c     advapi32:ADVAPI32.dll
 0002:00000010       __imp__RegSetValueExA@24   0040e010     advapi32:ADVAPI32.dll
 0002:00000014       __imp__RegCloseKey@4       0040e014     advapi32:ADVAPI32.dll
 0002:00000018       \177ADVAPI32_NULL_THUNK_DATA 0040e018     advapi32:ADVAPI32.dll
 0002:0000001c       __imp__InitializeSListHead@4 0040e01c     kernel32:KERNEL32.dll
 0002:00000020       __imp__GetCurrentProcessId@0 0040e020     kernel32:KERNEL32.dll
 0002:00000024       __imp__QueryPerformanceCounter@4 0040e024     kernel32:KERNEL32.dll
 0002:00000028       __imp__GetStartupInfoW@4   0040e028     kernel32:KERNEL32.dll
 0002:0000002c       __imp__IsDebuggerPresent@0 0040e02c     kernel32:KERNEL32.dll
 0002:00000030       __imp__GetModuleHandleW@4  0040e030     kernel32:KERNEL32.dll
 0002:00000034       __imp__CreateEventW@16     0040e034     kernel32:KERNEL32.dll
 0002:00000038       __imp__WaitForSingleObjectEx@12 0040e038     kernel32:KERNEL32.dll
 0002:0000003c       __imp__ResetEvent@4        0040e03c     kernel32:KERNEL32.dll
 0002:00000040       __imp__SetEvent@4          0040e040     kernel32:KERNEL32.dll
 0002:00000044       __imp__DeleteCriticalSection@4 0040e044     kernel32:KERNEL32.dll
 0002:00000048       __imp__InitializeCriticalSectionAndSpinCount@8 0040e048     kernel32:KERNEL32.dll
 0002:0000004c       __imp__LeaveCriticalSection@4 0040e04c     kernel32:KERNEL32.dll
 0002:00000050       __imp__EnterCriticalSection@4 0040e050     kernel32:KERNEL32.dll
 0002:00000054       __imp__CloseHandle@4       0040e054     kernel32:KERNEL32.dll
 0002:00000058       __imp__IsProcessorFeaturePresent@4 0040e058     kernel32:KERNEL32.dll
 0002:0000005c       __imp__TerminateProcess@8  0040e05c     kernel32:KERNEL32.dll
 0002:00000060       __imp__GetCurrentProcess@0 0040e060     kernel32:KERNEL32.dll
 0002:00000064       __imp__SetUnhandledExceptionFilter@4 0040e064     kernel32:KERNEL32.dll
 0002:00000068       __imp__UnhandledExceptionFilter@4 0040e068     kernel32:KERNEL32.dll
 0002:0000006c       __imp__GetCurrentThreadId@0 0040e06c     kernel32:KERNEL32.dll
 0002:00000070       __imp__FormatMessageA@28   0040e070     kernel32:KERNEL32.dll
 0002:00000074       __imp__GetSystemTimeAsFileTime@4 0040e074     kernel32:KERNEL32.dll
 0002:00000078       __imp__LoadLibraryA@4      0040e078     kernel32:KERNEL32.dll
 0002:0000007c       __imp__GetProcAddress@8    0040e07c     kernel32:KERNEL32.dll
 0002:00000080       __imp__FreeLibrary@4       0040e080     kernel32:KERNEL32.dll
 0002:00000084       __imp__GetLastError@0      0040e084     kernel32:KERNEL32.dll
 0002:00000088       \177KERNEL32_NULL_THUNK_DATA 0040e088     kernel32:KERNEL32.dll
 0002:0000008c       __imp_?_Xlength_error@std@@YAXPBD@Z 0040e08c     msvcprt:MSVCP140.dll
 0002:00000090       \177MSVCP140_NULL_THUNK_DATA 0040e090     msvcprt:MSVCP140.dll
 0002:00000094       __imp__CopyRect@8          0040e094     user32:USER32.dll
 0002:00000098       __imp__OffsetRect@12       0040e098     user32:USER32.dll
 0002:0000009c       __imp__GetDesktopWindow@0  0040e09c     user32:USER32.dll
 0002:000000a0       __imp__GetParent@4         0040e0a0     user32:USER32.dll
 0002:000000a4       __imp__WindowFromPoint@8   0040e0a4     user32:USER32.dll
 0002:000000a8       __imp__GetWindow@8         0040e0a8     user32:USER32.dll
 0002:000000ac       __imp__SetWindowsHookExA@16 0040e0ac     user32:USER32.dll
 0002:000000b0       __imp__UnhookWindowsHookEx@4 0040e0b0     user32:USER32.dll
 0002:000000b4       __imp__CallNextHookEx@16   0040e0b4     user32:USER32.dll
 0002:000000b8       __imp__IsDialogMessageA@8  0040e0b8     user32:USER32.dll
 0002:000000bc       __imp__GetCursorPos@4      0040e0bc     user32:USER32.dll
 0002:000000c0       __imp__GetTopWindow@4      0040e0c0     user32:USER32.dll
 0002:000000c4       __imp__GetWindowRect@8     0040e0c4     user32:USER32.dll
 0002:000000c8       __imp__SetWindowTextA@8    0040e0c8     user32:USER32.dll
 0002:000000cc       __imp__UpdateWindow@4      0040e0cc     user32:USER32.dll
 0002:000000d0       __imp__CheckMenuItem@12    0040e0d0     user32:USER32.dll
 0002:000000d4       __imp__GetMenu@4           0040e0d4     user32:USER32.dll
 0002:000000d8       __imp__GetSystemMetrics@4  0040e0d8     user32:USER32.dll
 0002:000000dc       __imp__TranslateAcceleratorA@12 0040e0dc     user32:USER32.dll
 0002:000000e0       __imp__LoadAcceleratorsA@8 0040e0e0     user32:USER32.dll
 0002:000000e4       __imp__EnableWindow@8      0040e0e4     user32:USER32.dll
 0002:000000e8       __imp__KillTimer@8         0040e0e8     user32:USER32.dll
 0002:000000ec       __imp__SetTimer@16         0040e0ec     user32:USER32.dll
 0002:000000f0       __imp__GetFocus@0          0040e0f0     user32:USER32.dll
 0002:000000f4       __imp__SetFocus@4          0040e0f4     user32:USER32.dll
 0002:000000f8       __imp__GetDlgCtrlID@4      0040e0f8     user32:USER32.dll
 0002:000000fc       __imp__GetDlgItemInt@16    0040e0fc     user32:USER32.dll
 0002:00000100       __imp__GetDlgItem@8        0040e100     user32:USER32.dll
 0002:00000104       __imp__EndDialog@8         0040e104     user32:USER32.dll
 0002:00000108       __imp__CreateDialogParamA@20 0040e108     user32:USER32.dll
 0002:0000010c       __imp__SetWindowPos@28     0040e10c     user32:USER32.dll
 0002:00000110       __imp__ShowWindow@8        0040e110     user32:USER32.dll
 0002:00000114       __imp__PostQuitMessage@4   0040e114     user32:USER32.dll
 0002:00000118       __imp__PostMessageA@16     0040e118     user32:USER32.dll
 0002:0000011c       __imp__DispatchMessageA@4  0040e11c     user32:USER32.dll
 0002:00000120       __imp__TranslateMessage@4  0040e120     user32:USER32.dll
 0002:00000124       __imp__GetMessageA@16      0040e124     user32:USER32.dll
 0002:00000128       __imp__wsprintfA           0040e128     user32:USER32.dll
 0002:0000012c       __imp__SetDlgItemTextA@12  0040e12c     user32:USER32.dll
 0002:00000130       __imp__RegisterWindowMessageA@4 0040e130     user32:USER32.dll
 0002:00000134       \177USER32_NULL_THUNK_DATA 0040e134     user32:USER32.dll
 0002:00000138       __imp__memcpy              0040e138     vcruntime:VCRUNTIME140.dll
 0002:0000013c       __imp__memset              0040e13c     vcruntime:VCRUNTIME140.dll
 0002:00000140       __imp__memmove             0040e140     vcruntime:VCRUNTIME140.dll
 0002:00000144       __imp___CxxThrowException@8 0040e144     vcruntime:VCRUNTIME140.dll
 0002:00000148       __imp____CxxFrameHandler3  0040e148     vcruntime:VCRUNTIME140.dll
 0002:0000014c       __imp____std_exception_copy 0040e14c     vcruntime:VCRUNTIME140.dll
 0002:00000150       __imp____std_exception_destroy 0040e150     vcruntime:VCRUNTIME140.dll
 0002:00000154       __imp___except_handler4_common 0040e154     vcruntime:VCRUNTIME140.dll
 0002:00000158       \177VCRUNTIME140_NULL_THUNK_DATA 0040e158     vcruntime:VCRUNTIME140.dll
 0002:0000015c       __imp__getenv              0040e15c     ucrt:api-ms-win-crt-environment-l1-1-0.dll
 0002:00000160       \177api-ms-win-crt-environment-l1-1-0_NULL_THUNK_DATA 0040e160     ucrt:api-ms-win-crt-environment-l1-1-0.dll
 0002:00000164       __imp___set_new_mode       0040e164     ucrt:api-ms-win-crt-heap-l1-1-0.dll
 0002:00000168       __imp__malloc              0040e168     ucrt:api-ms-win-crt-heap-l1-1-0.dll
 0002:0000016c       __imp___callnewh           0040e16c     ucrt:api-ms-win-crt-heap-l1-1-0.dll
 0002:00000170       __imp__free                0040e170     ucrt:api-ms-win-crt-heap-l1-1-0.dll
 0002:00000174       \177api-ms-win-crt-heap-l1-1-0_NULL_THUNK_DATA 0040e174     ucrt:api-ms-win-crt-heap-l1-1-0.dll
 0002:00000178       __imp___configthreadlocale 0040e178     ucrt:api-ms-win-crt-locale-l1-1-0.dll
 0002:0000017c       \177api-ms-win-crt-locale-l1-1-0_NULL_THUNK_DATA 0040e17c     ucrt:api-ms-win-crt-locale-l1-1-0.dll
 0002:00000180       __imp____setusermatherr    0040e180     ucrt:api-ms-win-crt-math-l1-1-0.dll
 0002:00000184       \177api-ms-win-crt-math-l1-1-0_NULL_THUNK_DATA 0040e184     ucrt:api-ms-win-crt-math-l1-1-0.dll
 0002:00000188       __imp___exit               0040e188     ucrt:api-ms-win-crt-runtime-l1-1-0.dll
 0002:0000018c       __imp__exit                0040e18c     ucrt:api-ms-win-crt-runtime-l1-1-0.dll
 0002:00000190       __imp___initterm_e         0040e190     ucrt:api-ms-win-crt-runtime-l1-1-0.dll
 0002:00000194       __imp__terminate           0040e194     ucrt:api-ms-win-crt-runtime-l1-1-0.dll
 0002:00000198       __imp___controlfp_s        0040e198     ucrt:api-ms-win-crt-runtime-l1-1-0.dll
 0002:0000019c       __imp___c_exit             0040e19c     ucrt:api-ms-win-crt-runtime-l1-1-0.dll
 0002:000001a0       __imp___register_thread_local_exe_atexit_callback 0040e1a0     ucrt:api-ms-win-crt-runtime-l1-1-0.dll
 0002:000001a4       __imp___configure_narrow_argv 0040e1a4     ucrt:api-ms-win-crt-runtime-l1-1-0.dll
 0002:000001a8       __imp___initialize_narrow_environment 0040e1a8     ucrt:api-ms-win-crt-runtime-l1-1-0.dll
 0002:000001ac       __imp___initialize_onexit_table 0040e1ac     ucrt:api-ms-win-crt-runtime-l1-1-0.dll
 0002:000001b0       __imp___register_onexit_function 0040e1b0     ucrt:api-ms-win-crt-runtime-l1-1-0.dll
 0002:000001b4       __imp___crt_atexit         0040e1b4     ucrt:api-ms-win-crt-runtime-l1-1-0.dll
 0002:000001b8       __imp___cexit              0040e1b8     ucrt:api-ms-win-crt-runtime-l1-1-0.dll
 0002:000001bc       __imp___seh_filter_exe     0040e1bc     ucrt:api-ms-win-crt-runtime-l1-1-0.dll
 0002:000001c0       __imp___set_app_type       0040e1c0     ucrt:api-ms-win-crt-runtime-l1-1-0.dll
 0002:000001c4       __imp___invalid_parameter_noinfo_noreturn 0040e1c4     ucrt:api-ms-win-crt-runtime-l1-1-0.dll
 0002:000001c8       __imp___get_narrow_winmain_command_line 0040e1c8     ucrt:api-ms-win-crt-runtime-l1-1-0.dll
 0002:000001cc       __imp___initterm           0040e1cc     ucrt:api-ms-win-crt-runtime-l1-1-0.dll
 0002:000001d0       \177api-ms-win-crt-runtime-l1-1-0_NULL_THUNK_DATA 0040e1d0     ucrt:api-ms-win-crt-runtime-l1-1-0.dll
 0002:000001d4       __imp__fclose              0040e1d4     ucrt:api-ms-win-crt-stdio-l1-1-0.dll
 0002:000001d8       __imp____stdio_common_vfwprintf 0040e1d8     ucrt:api-ms-win-crt-stdio-l1-1-0.dll
 0002:000001dc       __imp___set_fmode          0040e1dc     ucrt:api-ms-win-crt-stdio-l1-1-0.dll
 0002:000001e0       __imp____stdio_common_vsprintf 0040e1e0     ucrt:api-ms-win-crt-stdio-l1-1-0.dll
 0002:000001e4       __imp__fflush              0040e1e4     ucrt:api-ms-win-crt-stdio-l1-1-0.dll
 0002:000001e8       __imp__fopen               0040e1e8     ucrt:api-ms-win-crt-stdio-l1-1-0.dll
 0002:000001ec       __imp____stdio_common_vfprintf 0040e1ec     ucrt:api-ms-win-crt-stdio-l1-1-0.dll
 0002:000001f0       __imp____p__commode        0040e1f0     ucrt:api-ms-win-crt-stdio-l1-1-0.dll
 0002:000001f4       __imp____acrt_iob_func     0040e1f4     ucrt:api-ms-win-crt-stdio-l1-1-0.dll
 0002:000001f8       \177api-ms-win-crt-stdio-l1-1-0_NULL_THUNK_DATA 0040e1f8     ucrt:api-ms-win-crt-stdio-l1-1-0.dll
 0002:000001fc       __imp__strncat             0040e1fc     ucrt:api-ms-win-crt-string-l1-1-0.dll
 0002:00000200       __imp__strncpy             0040e200     ucrt:api-ms-win-crt-string-l1-1-0.dll
 0002:00000204       __imp__strlen              0040e204     ucrt:api-ms-win-crt-string-l1-1-0.dll
 0002:00000208       __imp__strcpy              0040e208     ucrt:api-ms-win-crt-string-l1-1-0.dll
 0002:0000020c       \177api-ms-win-crt-string-l1-1-0_NULL_THUNK_DATA 0040e20c     ucrt:api-ms-win-crt-string-l1-1-0.dll
 0002:00000210       __imp__asctime             0040e210     ucrt:api-ms-win-crt-time-l1-1-0.dll
 0002:00000214       __imp___localtime64        0040e214     ucrt:api-ms-win-crt-time-l1-1-0.dll
 0002:00000218       __imp___time64             0040e218     ucrt:api-ms-win-crt-time-l1-1-0.dll
 0002:0000021c       \177api-ms-win-crt-time-l1-1-0_NULL_THUNK_DATA 0040e21c     ucrt:api-ms-win-crt-time-l1-1-0.dll
 0002:00000220       ___guard_check_icall_fptr  0040e220     MSVCRT:guard_support.obj
 0002:00000224       ___xc_a                    0040e224     MSVCRT:initializers.obj
 0002:00000230       ___xc_z                    0040e230     MSVCRT:initializers.obj
 0002:00000234       ___xi_a                    0040e234     MSVCRT:initializers.obj
 0002:00000244       ___xi_z                    0040e244     MSVCRT:initializers.obj
 0002:00000248       ___xl_a                    0040e248     MSVCRT:tlssup.obj
 0002:0000024c       ___xl_z                    0040e24c     MSVCRT:tlssup.obj
 0002:00000250       ___xp_a                    0040e250     MSVCRT:initializers.obj
 0002:00000254       ___xp_z                    0040e254     MSVCRT:initializers.obj
 0002:00000258       ___xt_a                    0040e258     MSVCRT:initializers.obj
 0002:0000025c       ___xt_z                    0040e25c     MSVCRT:initializers.obj
 0002:00001944       ??_C@_0BB@MOGOBHAF@list?$DMT?$DO?5too?5long@ 0040f944     MessageHistory.obj
 0002:00001958       ??_C@_0BA@JFNIOLAK@string?5too?5long@ 0040f958     MessageHistory.obj
 0002:00002148       ??_C@_1EC@JIJBPKFM@?$AAa?$AAp?$AAi?$AA?9?$AAm?$AAs?$AA?9?$AAw?$AAi?$AAn?$AA?9?$AAc?$AAo?$AAr?$AAe@ 00410148     MSVCRT:thread_safe_statics.obj
 0002:0000218c       ??_C@_1BK@MGMFAEKH@?$AAk?$AAe?$AAr?$AAn?$AAe?$AAl?$AA3?$AA2?$AA?4?$AAd?$AAl?$AAl@ 0041018c     MSVCRT:thread_safe_statics.obj
 0002:000021a8       ??_C@_0BM@HLJJNPAH@InitializeConditionVariable@ 004101a8     MSVCRT:thread_safe_statics.obj
 0002:000021c4       ??_C@_0BJ@JEBJOJFJ@SleepConditionVariableCS@ 004101c4     MSVCRT:thread_safe_statics.obj
 0002:000021e0       ??_C@_0BJ@PGPPEPCC@WakeAllConditionVariable@ 004101e0     MSVCRT:thread_safe_statics.obj
 0002:00002200       ??_7exception@std@@6B@     00410200     MSVCRT:throw_bad_alloc.obj
 0002:00002208       ??_C@_0BC@EOODALEL@Unknown?5exception@ 00410208     MSVCRT:throw_bad_alloc.obj
 0002:00002220       ??_7bad_alloc@std@@6B@     00410220     MSVCRT:throw_bad_alloc.obj
 0002:00002228       ??_C@_0P@GHFPNOJB@bad?5allocation@ 00410228     MSVCRT:throw_bad_alloc.obj
 0002:0000223c       ??_7bad_array_new_length@std@@6B@ 0041023c     MSVCRT:throw_bad_alloc.obj
 0002:00002244       ??_C@_0BF@KINCDENJ@bad?5array?5new?5length@ 00410244     MSVCRT:throw_bad_alloc.obj
 0002:00002260       ??_7type_info@@6B@         00410260     MSVCRT:std_type_info_static.obj
 0002:000022e0       __load_config_used         004102e0     MSVCRT:loadcfg.obj
 0002:00002380       __tls_used                 00410380     MSVCRT:tlssup.obj
 0002:00002398       ??_R4exception@std@@6B@    00410398     MSVCRT:throw_bad_alloc.obj
 0002:000023ac       ??_R3exception@std@@8      004103ac     MSVCRT:throw_bad_alloc.obj
 0002:000023bc       ??_R2exception@std@@8      004103bc     MSVCRT:throw_bad_alloc.obj
 0002:000023c4       ??_R1A@?0A@EA@exception@std@@8 004103c4     MSVCRT:throw_bad_alloc.obj
 0002:000023e0       ??_R4bad_alloc@std@@6B@    004103e0     MSVCRT:throw_bad_alloc.obj
 0002:000023f4       ??_R3bad_alloc@std@@8      004103f4     MSVCRT:throw_bad_alloc.obj
 0002:00002404       ??_R2bad_alloc@std@@8      00410404     MSVCRT:throw_bad_alloc.obj
 0002:00002410       ??_R1A@?0A@EA@bad_alloc@std@@8 00410410     MSVCRT:throw_bad_alloc.obj
 0002:0000242c       ??_R4bad_array_new_length@std@@6B@ 0041042c     MSVCRT:throw_bad_alloc.obj
 0002:00002440       ??_R3bad_array_new_length@std@@8 00410440     MSVCRT:throw_bad_alloc.obj
 0002:00002450       ??_R2bad_array_new_length@std@@8 00410450     MSVCRT:throw_bad_alloc.obj
 0002:00002460       ??_R1A@?0A@EA@bad_array_new_length@std@@8 00410460     MSVCRT:throw_bad_alloc.obj
 0002:0000247c       ??_R4type_info@@6B@        0041047c     MSVCRT:std_type_info_static.obj
 0002:00002490       ??_R3type_info@@8          00410490     MSVCRT:std_type_info_static.obj
 0002:000024a0       ??_R2type_info@@8          004104a0     MSVCRT:std_type_info_static.obj
 0002:000024a8       ??_R1A@?0A@EA@type_info@@8 004104a8     MSVCRT:std_type_info_static.obj
 0002:000024d0       ___safe_se_handler_table   004104d0     <linker-defined>
 0002:000028a8       ___rtc_iaa                 004108a8     MSVCRT:initsect.obj
 0002:000028ac       ___rtc_izz                 004108ac     MSVCRT:initsect.obj
 0002:000028b0       ___rtc_taa                 004108b0     MSVCRT:initsect.obj
 0002:000028b4       ___rtc_tzz                 004108b4     MSVCRT:initsect.obj
 0002:000028b8       __tls_start                004108b8     MSVCRT:tlssup.obj
 0002:000028bc       __Init_thread_epoch        004108bc     MSVCRT:thread_safe_statics.obj
 0002:000028c0       __tls_end                  004108c0     MSVCRT:tlssup.obj
 0002:00002a5c       __TI2?AVbad_alloc@std@@    00410a5c     MSVCRT:throw_bad_alloc.obj
 0002:00002a6c       __CTA2?AVbad_alloc@std@@   00410a6c     MSVCRT:throw_bad_alloc.obj
 0002:00002a78       __CT??_R0?AVbad_alloc@std@@@8??0bad_alloc@std@@QAE@ABV01@@Z12 00410a78     MSVCRT:throw_bad_alloc.obj
 0002:00002a94       __CT??_R0?AVexception@std@@@8??0exception@std@@QAE@ABV01@@Z12 00410a94     MSVCRT:throw_bad_alloc.obj
 0002:00002ab0       __TI3?AVbad_array_new_length@std@@ 00410ab0     MSVCRT:throw_bad_alloc.obj
 0002:00002ac0       __CTA3?AVbad_array_new_length@std@@ 00410ac0     MSVCRT:throw_bad_alloc.obj
 0002:00002ad0       __CT??_R0?AVbad_array_new_length@std@@@8??0bad_array_new_length@std@@QAE@ABV01@@Z12 00410ad0     MSVCRT:throw_bad_alloc.obj
 0002:00002aec       __IMPORT_DESCRIPTOR_ADVAPI32 00410aec     advapi32:ADVAPI32.dll
 0002:00002b00       __IMPORT_DESCRIPTOR_USER32 00410b00     user32:USER32.dll
 0002:00002b14       __IMPORT_DESCRIPTOR_MSVCP140 00410b14     msvcprt:MSVCP140.dll
 0002:00002b28       __IMPORT_DESCRIPTOR_KERNEL32 00410b28     kernel32:KERNEL32.dll
 0002:00002b3c       __IMPORT_DESCRIPTOR_VCRUNTIME140 00410b3c     vcruntime:VCRUNTIME140.dll
 0002:00002b50       __IMPORT_DESCRIPTOR_api-ms-win-crt-string-l1-1-0 00410b50     ucrt:api-ms-win-crt-string-l1-1-0.dll
 0002:00002b64       __IMPORT_DESCRIPTOR_api-ms-win-crt-stdio-l1-1-0 00410b64     ucrt:api-ms-win-crt-stdio-l1-1-0.dll
 0002:00002b78       __IMPORT_DESCRIPTOR_api-ms-win-crt-environment-l1-1-0 00410b78     ucrt:api-ms-win-crt-environment-l1-1-0.dll
 0002:00002b8c       __IMPORT_DESCRIPTOR_api-ms-win-crt-time-l1-1-0 00410b8c     ucrt:api-ms-win-crt-time-l1-1-0.dll
 0002:00002ba0       __IMPORT_DESCRIPTOR_api-ms-win-crt-runtime-l1-1-0 00410ba0     ucrt:api-ms-win-crt-runtime-l1-1-0.dll
 0002:00002bb4       __IMPORT_DESCRIPTOR_api-ms-win-crt-heap-l1-1-0 00410bb4     ucrt:api-ms-win-crt-heap-l1-1-0.dll
 0002:00002bc8       __IMPORT_DESCRIPTOR_api-ms-win-crt-math-l1-1-0 00410bc8     ucrt:api-ms-win-crt-math-l1-1-0.dll
 0002:00002bdc       __IMPORT_DESCRIPTOR_api-ms-win-crt-locale-l1-1-0 00410bdc     ucrt:api-ms-win-crt-locale-l1-1-0.dll
 0002:00002bf0       __NULL_IMPORT_DESCRIPTOR   00410bf0     advapi32:ADVAPI32.dll
 0003:00000a68       ?sm_MaxMessages@MessageHistory@@2IA 00412a68     MessageHistory.obj
 0003:00000a6c       ?szAppName@@3PADA          00412a6c     jaccessinspector.obj
 0003:00000a90       ___security_cookie_complement 00412a90     MSVCRT:gs_cookie.obj
 0003:00000a94       ___security_cookie         00412a94     MSVCRT:gs_cookie.obj
 0003:00000a98       __fltused                  00412a98     MSVCRT:fltused.obj
 0003:00000a9c       ___scrt_native_dllmain_reason 00412a9c     MSVCRT:utility.obj
 0003:00000aa0       __Init_global_epoch        00412aa0     MSVCRT:thread_safe_statics.obj
 0003:00000aa4       ___isa_enabled             00412aa4     MSVCRT:cpu_disp.obj
 0003:00000ab0       ___scrt_default_matherr    00412ab0     MSVCRT:matherr.obj
 0003:00000ab4       ___scrt_ucrt_dll_is_in_use 00412ab4     MSVCRT:ucrt_stubs.obj
 0003:00000ab8       ??_R0?AVbad_alloc@std@@@8  00412ab8     MSVCRT:throw_bad_alloc.obj
 0003:00000ad4       ??_R0?AVexception@std@@@8  00412ad4     MSVCRT:throw_bad_alloc.obj
 0003:00000af0       ??_R0?AVbad_array_new_length@std@@@8 00412af0     MSVCRT:throw_bad_alloc.obj
 0003:00000b18       ??_R0?AVtype_info@@@8      00412b18     MSVCRT:std_type_info_static.obj
 0003:00000b40       _theAccessBridgeInitializedFlag 00412b40     AccessBridgeCalls.obj
 0003:00000b48       ?_OptionsStorage@?1??__local_stdio_printf_options@@9@4_KA 00412b48     AccessBridgeDebug.obj
 0003:00000c58       ?theFromJavaHelloMsgID@@3IA 00412c58     AccessBridgeMessages.obj
 0003:00000c5c       ?theFromWindowsHelloMsgID@@3IA 00412c5c     AccessBridgeMessages.obj
 0003:00000c60       ?g_LogStringCallback@@3P6GXPBD@ZA 00412c60     AccessInfo.obj
 0003:00000ca8       ?theDialogWindow@@3PAUHWND__@@A 00412ca8     jaccessinspector.obj
 0003:00000cac       ?theGoToDialogWindow@@3PAUHWND__@@A 00412cac     jaccessinspector.obj
 0003:00000cb0       ?theInstance@@3PAUHINSTANCE__@@A 00412cb0     jaccessinspector.obj
 0003:00000cb4       ?theAccessBridgeLoadedFlag@@3HA 00412cb4     jaccessinspector.obj
 0003:00000cb8       ?prevKbdHook@@3PAUHHOOK__@@A 00412cb8     jaccessinspector.obj
 0003:00000cbc       ?prevMouseHook@@3PAUHHOOK__@@A 00412cbc     jaccessinspector.obj
 0003:00000cc0       ?updateMouse@@3HA          00412cc0     jaccessinspector.obj
 0003:00000cc4       ?updateF1@@3HA             00412cc4     jaccessinspector.obj
 0003:00000cc8       ?updateF2@@3HA             00412cc8     jaccessinspector.obj
 0003:00000ccc       ?trackMouse@@3HA           00412ccc     jaccessinspector.obj
 0003:00000cd0       ?trackMouseExited@@3HA     00412cd0     jaccessinspector.obj
 0003:00000cd4       ?trackMouseClicked@@3HA    00412cd4     jaccessinspector.obj
 0003:00000cd8       ?trackMousePressed@@3HA    00412cd8     jaccessinspector.obj
 0003:00000cdc       ?trackMouseReleased@@3HA   00412cdc     jaccessinspector.obj
 0003:00000ce0       ?trackFocus@@3HA           00412ce0     jaccessinspector.obj
 0003:00000ce4       ?trackFocusLost@@3HA       00412ce4     jaccessinspector.obj
 0003:00000ce8       ?trackCaret@@3HA           00412ce8     jaccessinspector.obj
 0003:00000cec       ?trackShutdown@@3HA        00412cec     jaccessinspector.obj
 0003:00000cf0       ?trackMenuSelected@@3HA    00412cf0     jaccessinspector.obj
 0003:00000cf4       ?trackMenuDeselected@@3HA  00412cf4     jaccessinspector.obj
 0003:00000cf8       ?trackMenuCanceled@@3HA    00412cf8     jaccessinspector.obj
 0003:00000cfc       ?trackPopupVisible@@3HA    00412cfc     jaccessinspector.obj
 0003:00000d00       ?trackPopupInvisible@@3HA  00412d00     jaccessinspector.obj
 0003:00000d04       ?trackPopupCanceled@@3HA   00412d04     jaccessinspector.obj
 0003:00000d08       ?trackPropertyNameChange@@3HA 00412d08     jaccessinspector.obj
 0003:00000d0c       ?trackPropertyDescriptionChange@@3HA 00412d0c     jaccessinspector.obj
 0003:00000d10       ?trackPropertyStateChange@@3HA 00412d10     jaccessinspector.obj
 0003:00000d14       ?trackPropertyValueChange@@3HA 00412d14     jaccessinspector.obj
 0003:00000d18       ?trackPropertySelectionChange@@3HA 00412d18     jaccessinspector.obj
 0003:00000d1c       ?trackPropertyTextChange@@3HA 00412d1c     jaccessinspector.obj
 0003:00000d20       ?trackPropertyCaretChange@@3HA 00412d20     jaccessinspector.obj
 0003:00000d24       ?trackPropertyVisibleDataChange@@3HA 00412d24     jaccessinspector.obj
 0003:00000d28       ?trackPropertyChildChange@@3HA 00412d28     jaccessinspector.obj
 0003:00000d2c       ?trackPropertyActiveDescendentChange@@3HA 00412d2c     jaccessinspector.obj
 0003:00000d30       ?trackPropertyTableModelChange@@3HA 00412d30     jaccessinspector.obj
 0003:00000d34       ?logfile@@3PAU_iobuf@@A    00412d34     jaccessinspector.obj
 0003:00000d38       ?g_MessageHistory@@3VMessageHistory@@A 00412d38     jaccessinspector.obj
 0003:0000108c       ___scrt_current_native_startup_state 0041308c     MSVCRT:utility.obj
 0003:00001090       ___scrt_native_startup_lock 00413090     MSVCRT:utility.obj
 0003:000010d8       __tls_index                004130d8     MSVCRT:tlssup.obj
 0003:000010dc       ___isa_available           004130dc     MSVCRT:cpu_disp.obj
 0003:000010e0       ___favor                   004130e0     MSVCRT:cpu_disp.obj
 0003:000010e4       ___scrt_debugger_hook_flag 004130e4     MSVCRT:utility_desktop.obj
 0003:000010e8       ?__type_info_root_node@@3U__type_info_node@@A 004130e8     MSVCRT:tncleanup.obj
 0003:000010f0       ?_OptionsStorage@?1??__local_stdio_scanf_options@@9@4_KA 004130f0     MSVCRT:default_local_stdio_options.obj
 0003:00001100       _theAccessBridge           00413100     <common>
 0003:00001284       _theAccessBridgeInstance   00413284     <common>
 0003:00001288       ___dyn_tls_dtor_callback   00413288     <common>
 0003:0000128c       ___dyn_tls_init_callback   0041328c     <common>

 entry point at        0001:0000c296

 Static symbols

 0000:fffe8000       .debug$S                   00400000     kernel32:KERNEL32.dll
 0000:fffe8000       .debug$S                   00400000     user32:USER32.dll
 0000:fffe8000       .debug$S                   00400000     user32:USER32.dll
 0000:fffe8000       .debug$S                   00400000     user32:USER32.dll
 0000:fffe8000       .debug$S                   00400000     user32:USER32.dll
 0000:fffe8000       .debug$S                   00400000     user32:USER32.dll
 0000:fffe8000       .debug$S                   00400000     user32:USER32.dll
 0000:fffe8000       .debug$S                   00400000     advapi32:ADVAPI32.dll
 0000:fffe8000       .debug$S                   00400000     advapi32:ADVAPI32.dll
 0000:fffe8000       .debug$S                   00400000     advapi32:ADVAPI32.dll
 0000:fffe8000       .debug$S                   00400000     advapi32:ADVAPI32.dll
 0000:fffe8000       .debug$S                   00400000     advapi32:ADVAPI32.dll
 0000:fffe8000       .debug$S                   00400000     advapi32:ADVAPI32.dll
 0000:fffe8000       .debug$S                   00400000     ucrt:api-ms-win-crt-runtime-l1-1-0.dll
 0000:fffe8000       .debug$S                   00400000     ucrt:api-ms-win-crt-runtime-l1-1-0.dll
 0000:fffe8000       .debug$S                   00400000     ucrt:api-ms-win-crt-heap-l1-1-0.dll
 0000:fffe8000       .debug$S                   00400000     ucrt:api-ms-win-crt-stdio-l1-1-0.dll
 0000:fffe8000       .debug$S                   00400000     ucrt:api-ms-win-crt-heap-l1-1-0.dll
 0000:fffe8000       .debug$S                   00400000     ucrt:api-ms-win-crt-locale-l1-1-0.dll
 0000:fffe8000       .debug$S                   00400000     ucrt:api-ms-win-crt-runtime-l1-1-0.dll
 0000:fffe8000       .debug$S                   00400000     ucrt:api-ms-win-crt-runtime-l1-1-0.dll
 0000:fffe8000       .debug$S                   00400000     ucrt:api-ms-win-crt-stdio-l1-1-0.dll
 0000:fffe8000       .debug$S                   00400000     ucrt:api-ms-win-crt-runtime-l1-1-0.dll
 0000:fffe8000       .debug$S                   00400000     ucrt:api-ms-win-crt-runtime-l1-1-0.dll
 0000:fffe8000       .debug$S                   00400000     ucrt:api-ms-win-crt-runtime-l1-1-0.dll
 0000:fffe8000       .debug$S                   00400000     ucrt:api-ms-win-crt-runtime-l1-1-0.dll
 0000:fffe8000       .debug$S                   00400000     ucrt:api-ms-win-crt-runtime-l1-1-0.dll
 0000:fffe8000       .debug$S                   00400000     ucrt:api-ms-win-crt-math-l1-1-0.dll
 0000:fffe8000       .debug$S                   00400000     ucrt:api-ms-win-crt-runtime-l1-1-0.dll
 0000:fffe8000       .debug$S                   00400000     ucrt:api-ms-win-crt-runtime-l1-1-0.dll
 0000:fffe8000       .debug$S                   00400000     ucrt:api-ms-win-crt-runtime-l1-1-0.dll
 0000:fffe8000       .debug$S                   00400000     ucrt:api-ms-win-crt-runtime-l1-1-0.dll
 0000:fffe8000       .debug$S                   00400000     ucrt:api-ms-win-crt-runtime-l1-1-0.dll
 0000:fffe8000       .debug$S                   00400000     ucrt:api-ms-win-crt-runtime-l1-1-0.dll
 0000:fffe8000       .debug$S                   00400000     ucrt:api-ms-win-crt-runtime-l1-1-0.dll
 0000:fffe8000       .debug$S                   00400000     ucrt:api-ms-win-crt-runtime-l1-1-0.dll
 0000:fffe8000       .debug$S                   00400000     ucrt:api-ms-win-crt-runtime-l1-1-0.dll
 0000:fffe8000       .debug$S                   00400000     ucrt:api-ms-win-crt-runtime-l1-1-0.dll
 0000:fffe8000       .debug$S                   00400000     ucrt:api-ms-win-crt-runtime-l1-1-0.dll
 0000:fffe8000       .debug$S                   00400000     ucrt:api-ms-win-crt-heap-l1-1-0.dll
 0000:fffe8000       .debug$S                   00400000     ucrt:api-ms-win-crt-heap-l1-1-0.dll
 0000:fffe8000       .debug$S                   00400000     ucrt:api-ms-win-crt-runtime-l1-1-0.dll
 0000:fffe8000       .debug$S                   00400000     ucrt:api-ms-win-crt-time-l1-1-0.dll
 0000:fffe8000       .debug$S                   00400000     ucrt:api-ms-win-crt-time-l1-1-0.dll
 0000:fffe8000       .debug$S                   00400000     ucrt:api-ms-win-crt-time-l1-1-0.dll
 0000:fffe8000       .debug$S                   00400000     ucrt:api-ms-win-crt-stdio-l1-1-0.dll
 0000:fffe8000       .debug$S                   00400000     ucrt:api-ms-win-crt-stdio-l1-1-0.dll
 0000:fffe8000       .debug$S                   00400000     ucrt:api-ms-win-crt-string-l1-1-0.dll
 0000:fffe8000       .debug$S                   00400000     ucrt:api-ms-win-crt-environment-l1-1-0.dll
 0000:fffe8000       .debug$S                   00400000     ucrt:api-ms-win-crt-stdio-l1-1-0.dll
 0000:fffe8000       .debug$S                   00400000     ucrt:api-ms-win-crt-stdio-l1-1-0.dll
 0000:fffe8000       .debug$S                   00400000     ucrt:api-ms-win-crt-stdio-l1-1-0.dll
 0000:fffe8000       .debug$S                   00400000     ucrt:api-ms-win-crt-stdio-l1-1-0.dll
 0000:fffe8000       .debug$S                   00400000     ucrt:api-ms-win-crt-stdio-l1-1-0.dll
 0000:fffe8000       .debug$S                   00400000     ucrt:api-ms-win-crt-string-l1-1-0.dll
 0000:fffe8000       .debug$S                   00400000     ucrt:api-ms-win-crt-string-l1-1-0.dll
 0000:fffe8000       .debug$S                   00400000     ucrt:api-ms-win-crt-string-l1-1-0.dll
 0000:fffe8000       .debug$S                   00400000     user32:USER32.dll
 0000:fffe8000       .debug$S                   00400000     vcruntime:VCRUNTIME140.dll
 0000:fffe8000       .debug$S                   00400000     vcruntime:VCRUNTIME140.dll
 0000:fffe8000       .debug$S                   00400000     vcruntime:VCRUNTIME140.dll
 0000:fffe8000       .debug$S                   00400000     vcruntime:VCRUNTIME140.dll
 0000:fffe8000       .debug$S                   00400000     vcruntime:VCRUNTIME140.dll
 0000:fffe8000       .debug$S                   00400000     vcruntime:VCRUNTIME140.dll
 0000:fffe8000       .debug$S                   00400000     vcruntime:VCRUNTIME140.dll
 0000:fffe8000       .debug$S                   00400000     vcruntime:VCRUNTIME140.dll
 0000:fffe8000       .debug$S                   00400000     vcruntime:VCRUNTIME140.dll
 0000:fffe8000       .debug$S                   00400000     user32:USER32.dll
 0000:fffe8000       .debug$S                   00400000     user32:USER32.dll
 0000:fffe8000       .debug$S                   00400000     kernel32:KERNEL32.dll
 0000:fffe8000       .debug$S                   00400000     kernel32:KERNEL32.dll
 0000:fffe8000       .debug$S                   00400000     kernel32:KERNEL32.dll
 0000:fffe8000       .debug$S                   00400000     kernel32:KERNEL32.dll
 0000:fffe8000       .debug$S                   00400000     kernel32:KERNEL32.dll
 0000:fffe8000       .debug$S                   00400000     kernel32:KERNEL32.dll
 0000:fffe8000       .debug$S                   00400000     kernel32:KERNEL32.dll
 0000:fffe8000       .debug$S                   00400000     kernel32:KERNEL32.dll
 0000:fffe8000       .debug$S                   00400000     kernel32:KERNEL32.dll
 0000:fffe8000       .debug$S                   00400000     kernel32:KERNEL32.dll
 0000:fffe8000       .debug$S                   00400000     kernel32:KERNEL32.dll
 0000:fffe8000       .debug$S                   00400000     kernel32:KERNEL32.dll
 0000:fffe8000       .debug$S                   00400000     kernel32:KERNEL32.dll
 0000:fffe8000       .debug$S                   00400000     kernel32:KERNEL32.dll
 0000:fffe8000       .debug$S                   00400000     kernel32:KERNEL32.dll
 0000:fffe8000       .debug$S                   00400000     kernel32:KERNEL32.dll
 0000:fffe8000       .debug$S                   00400000     kernel32:KERNEL32.dll
 0000:fffe8000       .debug$S                   00400000     kernel32:KERNEL32.dll
 0000:fffe8000       .debug$S                   00400000     kernel32:KERNEL32.dll
 0000:fffe8000       .debug$S                   00400000     kernel32:KERNEL32.dll
 0000:fffe8000       .debug$S                   00400000     kernel32:KERNEL32.dll
 0000:fffe8000       .debug$S                   00400000     kernel32:KERNEL32.dll
 0000:fffe8000       .debug$S                   00400000     kernel32:KERNEL32.dll
 0000:fffe8000       .debug$S                   00400000     kernel32:KERNEL32.dll
 0000:fffe8000       .debug$S                   00400000     kernel32:KERNEL32.dll
 0000:fffe8000       .debug$S                   00400000     kernel32:KERNEL32.dll
 0000:fffe8000       .debug$S                   00400000     user32:USER32.dll
 0000:fffe8000       .debug$S                   00400000     msvcprt:MSVCP140.dll
 0000:fffe8000       .debug$S                   00400000     user32:USER32.dll
 0000:fffe8000       .debug$S                   00400000     user32:USER32.dll
 0000:fffe8000       .debug$S                   00400000     user32:USER32.dll
 0000:fffe8000       .debug$S                   00400000     user32:USER32.dll
 0000:fffe8000       .debug$S                   00400000     user32:USER32.dll
 0000:fffe8000       .debug$S                   00400000     user32:USER32.dll
 0000:fffe8000       .debug$S                   00400000     user32:USER32.dll
 0000:fffe8000       .debug$S                   00400000     user32:USER32.dll
 0000:fffe8000       .debug$S                   00400000     user32:USER32.dll
 0000:fffe8000       .debug$S                   00400000     user32:USER32.dll
 0000:fffe8000       .debug$S                   00400000     user32:USER32.dll
 0000:fffe8000       .debug$S                   00400000     user32:USER32.dll
 0000:fffe8000       .debug$S                   00400000     user32:USER32.dll
 0000:fffe8000       .debug$S                   00400000     user32:USER32.dll
 0000:fffe8000       .debug$S                   00400000     user32:USER32.dll
 0000:fffe8000       .debug$S                   00400000     user32:USER32.dll
 0000:fffe8000       .debug$S                   00400000     user32:USER32.dll
 0000:fffe8000       .debug$S                   00400000     user32:USER32.dll
 0000:fffe8000       .debug$S                   00400000     user32:USER32.dll
 0000:fffe8000       .debug$S                   00400000     user32:USER32.dll
 0000:fffe8000       .debug$S                   00400000     user32:USER32.dll
 0000:fffe8000       .debug$S                   00400000     user32:USER32.dll
 0000:fffe8000       .debug$S                   00400000     user32:USER32.dll
 0000:fffe8000       .debug$S                   00400000     user32:USER32.dll
 0000:fffe8000       .debug$S                   00400000     user32:USER32.dll
 0000:fffe8000       .debug$S                   00400000     user32:USER32.dll
 0000:fffe8000       .debug$S                   00400000     user32:USER32.dll
 0000:fffe8000       .debug$S                   00400000     user32:USER32.dll
 0000:fffe8000       .debug$S                   00400000     user32:USER32.dll
 0000:fffe8000       .debug$S                   00400000     user32:USER32.dll
 0001:00000000       ??__Eg_MessageHistory@@YAXXZ 00401000 f   jaccessinspector.obj
 0001:000049b0       _localtime                 004059b0 f   AccessInfo.obj
 0001:000049d0       _time                      004059d0 f   AccessInfo.obj
 0001:000051ef       __catch$??$_Buynode@V?$basic_string@DU?$char_traits@D@std@@V?$allocator@D@2@@std@@@?$_List_buy@V?$basic_string@DU?$char_traits@D@std@@V?$allocator@D@2@@std@@V?$allocator@V?$basic_string@DU?$char_traits@D@std@@V?$allocator@D@2@@std@@@2@@std@@QAEPAU?$_List_node@V?$basic_string@DU?$char_traits@D@std@@V?$allocator@D@2@@std@@PAX@1@PAU21@0$$QAV?$basic_string@DU?$char_traits@D@std@@V?$allocator@D@2@@1@@Z$0 004061ef f i MessageHistory.obj
 0001:00005bb6       __catch$?_Buynode0@?$_List_alloc@U?$_List_base_types@V?$basic_string@DU?$char_traits@D@std@@V?$allocator@D@2@@std@@V?$allocator@V?$basic_string@DU?$char_traits@D@std@@V?$allocator@D@2@@std@@@2@@std@@@std@@QAEPAU?$_List_node@V?$basic_string@DU?$char_traits@D@std@@V?$allocator@D@2@@std@@PAX@2@PAU32@0@Z$0 00406bb6 f i MessageHistory.obj
 0001:000081c8       $LN133                     004091c8     jaccessinspector.obj
 0001:000081dc       $LN131                     004091dc     jaccessinspector.obj
 0001:00008200       $LN134                     00409200     jaccessinspector.obj
 0001:00008210       $LN135                     00409210     jaccessinspector.obj
 0001:00008248       $LN132                     00409248     jaccessinspector.obj
 0001:00008314       $LN136                     00409314     jaccessinspector.obj
 0001:0000ba60       $$000000                   0040ca60     MSVCRT:ulldiv.obj
 0001:0000bae0       $$000000                   0040cae0     MSVCRT:chkstk.obj
 0001:0000bb4b       ?find_pe_section@@YAPAU_IMAGE_SECTION_HEADER@@QAEI@Z 0040cb4b f   MSVCRT:utility.obj
 0001:0000bdc8       ?__scrt_initialize_thread_safe_statics@@YAHXZ 0040cdc8 f   MSVCRT:thread_safe_statics.obj
 0001:0000be0c       ?__scrt_initialize_thread_safe_statics_platform_specific@@YAXXZ 0040ce0c f   MSVCRT:thread_safe_statics.obj
 0001:0000befb       ?__scrt_uninitialize_thread_safe_statics@@YAXXZ 0040cefb f   MSVCRT:thread_safe_statics.obj
 0001:0000c055       ?pre_c_initialization@@YAHXZ 0040d055 f   MSVCRT:exe_winmain.obj
 0001:0000c100       ?post_pgo_initialization@@YAHXZ 0040d100 f   MSVCRT:exe_winmain.obj
 0001:0000c108       ?pre_cpp_initialization@@YAXXZ 0040d108 f   MSVCRT:exe_winmain.obj
 0001:0000c11a       ?__scrt_common_main_seh@@YAHXZ 0040d11a f   MSVCRT:exe_winmain.obj
 0001:0000c750       $$000000                   0040d750     MSVCRT:sehprolg4.obj
 0001:0000c7cf       ___get_entropy             0040d7cf f   MSVCRT:gs_support.obj
 0001:0000ca40       __unwindfunclet$?AddMessage@MessageHistory@@QAEXPBD@Z$0 0040da40 f   MessageHistory.obj
 0001:0000ca48       __ehhandler$?AddMessage@MessageHistory@@QAEXPBD@Z 0040da48 f   MessageHistory.obj
 0001:0000ca70       __ehhandler$??$_Buynode@V?$basic_string@DU?$char_traits@D@std@@V?$allocator@D@2@@std@@@?$_List_buy@V?$basic_string@DU?$char_traits@D@std@@V?$allocator@D@2@@std@@V?$allocator@V?$basic_string@DU?$char_traits@D@std@@V?$allocator@D@2@@std@@@2@@std@@QAEPAU?$_List_node@V?$basic_string@DU?$char_traits@D@std@@V?$allocator@D@2@@std@@PAX@1@PAU21@0$$QAV?$basic_string@DU?$char_traits@D@std@@V?$allocator@D@2@@1@@Z 0040da70 f   MessageHistory.obj
 0001:0000ca90       __ehhandler$?c_str@?$basic_string@DU?$char_traits@D@std@@V?$allocator@D@2@@std@@QBEPBDXZ 0040da90 f   MessageHistory.obj
 0001:0000ca90       __ehhandler$?end@?$list@V?$basic_string@DU?$char_traits@D@std@@V?$allocator@D@2@@std@@V?$allocator@V?$basic_string@DU?$char_traits@D@std@@V?$allocator@D@2@@std@@@2@@std@@QAE?AV?$_List_iterator@V?$_List_val@U?$_List_simple_types@V?$basic_string@DU?$char_traits@D@std@@V?$allocator@D@2@@std@@@std@@@std@@@2@XZ 0040da90 f   MessageHistory.obj
 0001:0000ca90       __ehhandler$?_Make_iter@?$list@V?$basic_string@DU?$char_traits@D@std@@V?$allocator@D@2@@std@@V?$allocator@V?$basic_string@DU?$char_traits@D@std@@V?$allocator@D@2@@std@@@2@@std@@QBE?AV?$_List_iterator@V?$_List_val@U?$_List_simple_types@V?$basic_string@DU?$char_traits@D@std@@V?$allocator@D@2@@std@@@std@@@std@@@2@V?$_List_const_iterator@V?$_List_val@U?$_List_simple_types@V?$basic_string@DU?$char_traits@D@std@@V?$allocator@D@2@@std@@@std@@@std@@@2@@Z 0040da90 f   MessageHistory.obj
 0001:0000ca90       __ehhandler$?begin@?$list@V?$basic_string@DU?$char_traits@D@std@@V?$allocator@D@2@@std@@V?$allocator@V?$basic_string@DU?$char_traits@D@std@@V?$allocator@D@2@@std@@@2@@std@@QAE?AV?$_List_iterator@V?$_List_val@U?$_List_simple_types@V?$basic_string@DU?$char_traits@D@std@@V?$allocator@D@2@@std@@@std@@@std@@@2@XZ 0040da90 f   MessageHistory.obj
 0001:0000ca90       __ehhandler$??1?$list@V?$basic_string@DU?$char_traits@D@std@@V?$allocator@D@2@@std@@V?$allocator@V?$basic_string@DU?$char_traits@D@std@@V?$allocator@D@2@@std@@@2@@std@@QAE@XZ 0040da90 f   jaccessinspector.obj
 0001:0000ca90       __ehhandler$??1?$basic_string@DU?$char_traits@D@std@@V?$allocator@D@2@@std@@QAE@XZ 0040da90 f   MessageHistory.obj
 0001:0000ca90       __ehhandler$??1?$_List_alloc@U?$_List_base_types@V?$basic_string@DU?$char_traits@D@std@@V?$allocator@D@2@@std@@V?$allocator@V?$basic_string@DU?$char_traits@D@std@@V?$allocator@D@2@@std@@@2@@std@@@std@@QAE@XZ 0040da90 f   jaccessinspector.obj
 0001:0000ca90       __ehhandler$??$_Freenode0@V?$allocator@U?$_List_node@V?$basic_string@DU?$char_traits@D@std@@V?$allocator@D@2@@std@@PAX@std@@@std@@@?$_List_node@V?$basic_string@DU?$char_traits@D@std@@V?$allocator@D@2@@std@@PAX@std@@SAXAAV?$allocator@U?$_List_node@V?$basic_string@DU?$char_traits@D@std@@V?$allocator@D@2@@std@@PAX@std@@@1@PAU01@@Z 0040da90 f   MessageHistory.obj
 0001:0000cab0       __ehhandler$??0?$basic_string@DU?$char_traits@D@std@@V?$allocator@D@2@@std@@QAE@$$QAV01@@Z 0040dab0 f   MessageHistory.obj
 0001:0000cad0       __unwindfunclet$??0?$basic_string@DU?$char_traits@D@std@@V?$allocator@D@2@@std@@QAE@QBD@Z$0 0040dad0 f   MessageHistory.obj
 0001:0000cad8       __ehhandler$??0?$basic_string@DU?$char_traits@D@std@@V?$allocator@D@2@@std@@QAE@QBD@Z 0040dad8 f   MessageHistory.obj
 0001:0000cb00       __ehhandler$?clear@?$list@V?$basic_string@DU?$char_traits@D@std@@V?$allocator@D@2@@std@@V?$allocator@V?$basic_string@DU?$char_traits@D@std@@V?$allocator@D@2@@std@@@2@@std@@QAEXXZ 0040db00 f   MessageHistory.obj
 0001:0000cb00       __ehhandler$?_Assign_rv_contents_with_alloc_always_equal@?$basic_string@DU?$char_traits@D@std@@V?$allocator@D@2@@std@@QAEX$$QAV12@U?$integral_constant@_N$00@2@@Z 0040db00 f   MessageHistory.obj
 0001:0000cb20       __ehhandler$?_Buynode0@?$_List_alloc@U?$_List_base_types@V?$basic_string@DU?$char_traits@D@std@@V?$allocator@D@2@@std@@V?$allocator@V?$basic_string@DU?$char_traits@D@std@@V?$allocator@D@2@@std@@@2@@std@@@std@@QAEPAU?$_List_node@V?$basic_string@DU?$char_traits@D@std@@V?$allocator@D@2@@std@@PAX@2@PAU32@0@Z 0040db20 f   MessageHistory.obj
 0001:0000cb40       __unwindfunclet$??0MessageHistory@@QAE@XZ$0 0040db40 f   jaccessinspector.obj
 0001:0000cb48       __ehhandler$??0MessageHistory@@QAE@XZ 0040db48 f   jaccessinspector.obj
 0001:0000cb63       __ehhandler$?__scrt_initialize_thread_safe_statics_platform_specific@@YAXXZ 0040db63 f   MSVCRT:thread_safe_statics.obj
 0001:0000cb80       ??__Fg_MessageHistory@@YAXXZ 0040db80 f   jaccessinspector.obj
 0002:00000228       ?pre_cpp_initializer@@3P6AXXZA 0040e228     MSVCRT:exe_winmain.obj
 0002:0000022c       ?g_MessageHistory$initializer$@@3P6AXXZA 0040e22c     jaccessinspector.obj
 0002:00000238       ?pre_c_initializer@@3P6AHXZA 0040e238     MSVCRT:exe_winmain.obj
 0002:0000023c       ?post_pgo_initializer@@3P6AHXZA 0040e23c     MSVCRT:exe_winmain.obj
 0002:00000240       ?__scrt_initialize_tss_var@@3P6AHXZA 0040e240     MSVCRT:thread_safe_statics.obj
 0002:00000260       $SG45876                   0040e260     AccessBridgeDebug.obj
 0002:0000027c       $SG45878                   0040e27c     AccessBridgeDebug.obj
 0002:00000284       $SG45879                   0040e284     AccessBridgeDebug.obj
 0002:00000288       $SG45881                   0040e288     AccessBridgeDebug.obj
 0002:00000290       $SG45882                   0040e290     AccessBridgeDebug.obj
 0002:000002a8       $SG45909                   0040e2a8     AccessBridgeDebug.obj
 0002:000002c4       $SG45910                   0040e2c4     AccessBridgeDebug.obj
 0002:000002d0       $SG45912                   0040e2d0     AccessBridgeDebug.obj
 0002:000002d4       $SG45954                   0040e2d4     AccessBridgeDebug.obj
 0002:000002dc       $SG45955                   0040e2dc     AccessBridgeDebug.obj
 0002:000002e0       $SG45971                   0040e2e0     AccessBridgeDebug.obj
 0002:000002e8       $SG45972                   0040e2e8     AccessBridgeDebug.obj
 0002:000002ec       $SG46014                   0040e2ec     AccessBridgeDebug.obj
 0002:000002f4       $SG46015                   0040e2f4     AccessBridgeDebug.obj
 0002:000002f8       $SG46031                   0040e2f8     AccessBridgeDebug.obj
 0002:00000300       $SG46032                   0040e300     AccessBridgeDebug.obj
 0002:00000304       $SG40743                   0040e304     AccessBridgeMessages.obj
 0002:00000320       $SG40744                   0040e320     AccessBridgeMessages.obj
 0002:00000340       $SG50163                   0040e340     AccessInfo.obj
 0002:00000344       $SG50165                   0040e344     AccessInfo.obj
 0002:00000348       $SG50168                   0040e348     AccessInfo.obj
 0002:00000354       $SG50213                   0040e354     AccessInfo.obj
 0002:00000380       $SG50214                   0040e380     AccessInfo.obj
 0002:00000384       $SG50215                   0040e384     AccessInfo.obj
 0002:00000388       $SG50233                   0040e388     AccessInfo.obj
 0002:0000038c       $SG50375                   0040e38c     AccessInfo.obj
 0002:000003b4       $SG50376                   0040e3b4     AccessInfo.obj
 0002:000003cc       $SG50377                   0040e3cc     AccessInfo.obj
 0002:000003f4       $SG50378                   0040e3f4     AccessInfo.obj
 0002:00000420       $SG50379                   0040e420     AccessInfo.obj
 0002:0000044c       $SG50380                   0040e44c     AccessInfo.obj
 0002:0000047c       $SG50384                   0040e47c     AccessInfo.obj
 0002:000004a8       $SG50385                   0040e4a8     AccessInfo.obj
 0002:000004cc       $SG50388                   0040e4cc     AccessInfo.obj
 0002:000004e8       $SG50389                   0040e4e8     AccessInfo.obj
 0002:000004ec       $SG50390                   0040e4ec     AccessInfo.obj
 0002:00000500       $SG50393                   0040e500     AccessInfo.obj
 0002:00000524       $SG50394                   0040e524     AccessInfo.obj
 0002:00000540       $SG50395                   0040e540     AccessInfo.obj
 0002:00000558       $SG50396                   0040e558     AccessInfo.obj
 0002:0000056c       $SG50397                   0040e56c     AccessInfo.obj
 0002:00000590       $SG50398                   0040e590     AccessInfo.obj
 0002:000005a4       $SG50399                   0040e5a4     AccessInfo.obj
 0002:000005c8       $SG50400                   0040e5c8     AccessInfo.obj
 0002:000005e4       $SG50401                   0040e5e4     AccessInfo.obj
 0002:00000600       $SG50402                   0040e600     AccessInfo.obj
 0002:0000062c       $SG50405                   0040e62c     AccessInfo.obj
 0002:00000650       $SG50408                   0040e650     AccessInfo.obj
 0002:00000690       $SG50411                   0040e690     AccessInfo.obj
 0002:000006b4       $SG50412                   0040e6b4     AccessInfo.obj
 0002:000006d8       $SG50413                   0040e6d8     AccessInfo.obj
 0002:000006fc       $SG50416                   0040e6fc     AccessInfo.obj
 0002:0000070c       $SG50419                   0040e70c     AccessInfo.obj
 0002:00000740       $SG50420                   0040e740     AccessInfo.obj
 0002:00000758       $SG50423                   0040e758     AccessInfo.obj
 0002:0000077c       $SG50424                   0040e77c     AccessInfo.obj
 0002:0000079c       $SG50425                   0040e79c     AccessInfo.obj
 0002:000007b4       $SG50428                   0040e7b4     AccessInfo.obj
 0002:000007dc       $SG50429                   0040e7dc     AccessInfo.obj
 0002:00000804       $SG50433                   0040e804     AccessInfo.obj
 0002:00000828       $SG50437                   0040e828     AccessInfo.obj
 0002:0000084c       $SG50438                   0040e84c     AccessInfo.obj
 0002:0000086c       $SG50439                   0040e86c     AccessInfo.obj
 0002:0000088c       $SG50441                   0040e88c     AccessInfo.obj
 0002:000008b4       $SG50443                   0040e8b4     AccessInfo.obj
 0002:000008d0       $SG50446                   0040e8d0     AccessInfo.obj
 0002:00000914       $SG50449                   0040e914     AccessInfo.obj
 0002:00000950       $SG50452                   0040e950     AccessInfo.obj
 0002:00000974       $SG50453                   0040e974     AccessInfo.obj
 0002:00000994       $SG50454                   0040e994     AccessInfo.obj
 0002:000009b4       $SG50455                   0040e9b4     AccessInfo.obj
 0002:000009e0       $SG50457                   0040e9e0     AccessInfo.obj
 0002:00000a00       $SG50458                   0040ea00     AccessInfo.obj
 0002:00000a24       $SG50459                   0040ea24     AccessInfo.obj
 0002:00000a48       $SG50460                   0040ea48     AccessInfo.obj
 0002:00000a6c       $SG50462                   0040ea6c     AccessInfo.obj
 0002:00000a88       $SG50463                   0040ea88     AccessInfo.obj
 0002:00000aa4       $SG50464                   0040eaa4     AccessInfo.obj
 0002:00000ac4       $SG50465                   0040eac4     AccessInfo.obj
 0002:00000ae0       $SG50466                   0040eae0     AccessInfo.obj
 0002:00000af8       $SG50468                   0040eaf8     AccessInfo.obj
 0002:00000b14       $SG50469                   0040eb14     AccessInfo.obj
 0002:00000b34       $SG50470                   0040eb34     AccessInfo.obj
 0002:00000b50       $SG50473                   0040eb50     AccessInfo.obj
 0002:00000b74       $SG50475                   0040eb74     AccessInfo.obj
 0002:00000b9c       $SG50476                   0040eb9c     AccessInfo.obj
 0002:00000bbc       $SG50477                   0040ebbc     AccessInfo.obj
 0002:00000bd8       $SG50478                   0040ebd8     AccessInfo.obj
 0002:00000bfc       $SG50481                   0040ebfc     AccessInfo.obj
 0002:00000c28       $SG50484                   0040ec28     AccessInfo.obj
 0002:00000c4c       $SG50485                   0040ec4c     AccessInfo.obj
 0002:00000c6c       $SG50486                   0040ec6c     AccessInfo.obj
 0002:00000c8c       $SG50488                   0040ec8c     AccessInfo.obj
 0002:00000cb0       $SG50490                   0040ecb0     AccessInfo.obj
 0002:00000ccc       $SG50492                   0040eccc     AccessInfo.obj
 0002:00000ce8       $SG50494                   0040ece8     AccessInfo.obj
 0002:00000d04       $SG50498                   0040ed04     AccessInfo.obj
 0002:00000d2c       $SG50499                   0040ed2c     AccessInfo.obj
 0002:00000d48       $SG50500                   0040ed48     AccessInfo.obj
 0002:00000d6c       $SG50501                   0040ed6c     AccessInfo.obj
 0002:00000d90       $SG50502                   0040ed90     AccessInfo.obj
 0002:00000db4       $SG50503                   0040edb4     AccessInfo.obj
 0002:00000dd0       $SG50504                   0040edd0     AccessInfo.obj
 0002:00000df0       $SG50507                   0040edf0     AccessInfo.obj
 0002:00000e1c       $SG50508                   0040ee1c     AccessInfo.obj
 0002:00000e48       $SG50509                   0040ee48     AccessInfo.obj
 0002:00000e5c       $SG50510                   0040ee5c     AccessInfo.obj
 0002:00000e74       $SG50511                   0040ee74     AccessInfo.obj
 0002:00000e90       $SG50512                   0040ee90     AccessInfo.obj
 0002:00000ea8       $SG50515                   0040eea8     AccessInfo.obj
 0002:00000eec       $SG50518                   0040eeec     AccessInfo.obj
 0002:00000f10       $SG50519                   0040ef10     AccessInfo.obj
 0002:00000f24       $SG50520                   0040ef24     AccessInfo.obj
 0002:00000f38       $SG50523                   0040ef38     AccessInfo.obj
 0002:00000f68       $SG50524                   0040ef68     AccessInfo.obj
 0002:00000f90       $SG50525                   0040ef90     AccessInfo.obj
 0002:00000fb4       $SG50526                   0040efb4     AccessInfo.obj
 0002:00000fdc       $SG50527                   0040efdc     AccessInfo.obj
 0002:00000ffc       $SG50530                   0040effc     AccessInfo.obj
 0002:00001030       $SG50531                   0040f030     AccessInfo.obj
 0002:00001048       $SG50532                   0040f048     AccessInfo.obj
 0002:0000104c       $SG50535                   0040f04c     AccessInfo.obj
 0002:00001078       $SG50536                   0040f078     AccessInfo.obj
 0002:0000109c       $SG50537                   0040f09c     AccessInfo.obj
 0002:000010b0       $SG50538                   0040f0b0     AccessInfo.obj
 0002:000010c8       $SG50539                   0040f0c8     AccessInfo.obj
 0002:000010e4       $SG50540                   0040f0e4     AccessInfo.obj
 0002:000010fc       $SG50543                   0040f0fc     AccessInfo.obj
 0002:00001128       $SG50546                   0040f128     AccessInfo.obj
 0002:0000114c       $SG50547                   0040f14c     AccessInfo.obj
 0002:00001160       $SG50548                   0040f160     AccessInfo.obj
 0002:00001174       $SG50550                   0040f174     AccessInfo.obj
 0002:00001198       $SG50552                   0040f198     AccessInfo.obj
 0002:000011c0       $SG50553                   0040f1c0     AccessInfo.obj
 0002:000011e0       $SG50554                   0040f1e0     AccessInfo.obj
 0002:000011f8       $SG50556                   0040f1f8     AccessInfo.obj
 0002:0000121c       $SG50557                   0040f21c     AccessInfo.obj
 0002:0000123c       $SG50558                   0040f23c     AccessInfo.obj
 0002:00001258       $SG50559                   0040f258     AccessInfo.obj
 0002:0000127c       $SG50561                   0040f27c     AccessInfo.obj
 0002:000012b8       $SG50564                   0040f2b8     AccessInfo.obj
 0002:000012d8       $SG50566                   0040f2d8     AccessInfo.obj
 0002:000012f4       $SG50567                   0040f2f4     AccessInfo.obj
 0002:0000130c       $SG50568                   0040f30c     AccessInfo.obj
 0002:00001328       $SG50570                   0040f328     AccessInfo.obj
 0002:00001330       $SG50571                   0040f330     AccessInfo.obj
 0002:0000133c       $SG50572                   0040f33c     AccessInfo.obj
 0002:0000135c       $SG50573                   0040f35c     AccessInfo.obj
 0002:00001364       $SG50574                   0040f364     AccessInfo.obj
 0002:00001370       $SG50575                   0040f370     AccessInfo.obj
 0002:00001378       $SG50576                   0040f378     AccessInfo.obj
 0002:00001384       $SG50577                   0040f384     AccessInfo.obj
 0002:00001394       $SG50578                   0040f394     AccessInfo.obj
 0002:0000139c       $SG50579                   0040f39c     AccessInfo.obj
 0002:000013ac       $SG50580                   0040f3ac     AccessInfo.obj
 0002:000013c0       $SG50581                   0040f3c0     AccessInfo.obj
 0002:000013c8       $SG50582                   0040f3c8     AccessInfo.obj
 0002:000013d4       $SG50583                   0040f3d4     AccessInfo.obj
 0002:000013e4       $SG50584                   0040f3e4     AccessInfo.obj
 0002:000013ec       $SG50585                   0040f3ec     AccessInfo.obj
 0002:000013f8       $SG50586                   0040f3f8     AccessInfo.obj
 0002:00001408       $SG50587                   0040f408     AccessInfo.obj
 0002:00001410       $SG50588                   0040f410     AccessInfo.obj
 0002:00001434       $SG50589                   0040f434     AccessInfo.obj
 0002:00001458       $SG50590                   0040f458     AccessInfo.obj
 0002:00001474       $SG50591                   0040f474     AccessInfo.obj
 0002:00001490       $SG50592                   0040f490     AccessInfo.obj
 0002:000014b4       $SG50593                   0040f4b4     AccessInfo.obj
 0002:000014d0       $SG50594                   0040f4d0     AccessInfo.obj
 0002:000014ec       $SG50595                   0040f4ec     AccessInfo.obj
 0002:00001508       $SG50596                   0040f508     AccessInfo.obj
 0002:00001524       $SG50597                   0040f524     AccessInfo.obj
 0002:00001540       $SG50598                   0040f540     AccessInfo.obj
 0002:00001568       $SG50601                   0040f568     AccessInfo.obj
 0002:00001588       $SG50602                   0040f588     AccessInfo.obj
 0002:000015b4       $SG50603                   0040f5b4     AccessInfo.obj
 0002:000015d0       $SG50605                   0040f5d0     AccessInfo.obj
 0002:00001608       $SG50607                   0040f608     AccessInfo.obj
 0002:00001644       $SG50610                   0040f644     AccessInfo.obj
 0002:00001664       $SG50612                   0040f664     AccessInfo.obj
 0002:00001680       $SG50613                   0040f680     AccessInfo.obj
 0002:00001698       $SG50614                   0040f698     AccessInfo.obj
 0002:000016b4       $SG50616                   0040f6b4     AccessInfo.obj
 0002:000016bc       $SG50617                   0040f6bc     AccessInfo.obj
 0002:000016c8       $SG50618                   0040f6c8     AccessInfo.obj
 0002:000016e8       $SG50619                   0040f6e8     AccessInfo.obj
 0002:000016f0       $SG50620                   0040f6f0     AccessInfo.obj
 0002:000016fc       $SG50621                   0040f6fc     AccessInfo.obj
 0002:00001704       $SG50622                   0040f704     AccessInfo.obj
 0002:00001710       $SG50623                   0040f710     AccessInfo.obj
 0002:00001720       $SG50624                   0040f720     AccessInfo.obj
 0002:00001728       $SG50625                   0040f728     AccessInfo.obj
 0002:00001738       $SG50626                   0040f738     AccessInfo.obj
 0002:0000174c       $SG50627                   0040f74c     AccessInfo.obj
 0002:00001754       $SG50628                   0040f754     AccessInfo.obj
 0002:00001760       $SG50629                   0040f760     AccessInfo.obj
 0002:00001770       $SG50630                   0040f770     AccessInfo.obj
 0002:00001778       $SG50631                   0040f778     AccessInfo.obj
 0002:00001784       $SG50632                   0040f784     AccessInfo.obj
 0002:00001794       $SG50633                   0040f794     AccessInfo.obj
 0002:0000179c       $SG50634                   0040f79c     AccessInfo.obj
 0002:000017c0       $SG50635                   0040f7c0     AccessInfo.obj
 0002:000017e4       $SG50636                   0040f7e4     AccessInfo.obj
 0002:00001800       $SG50637                   0040f800     AccessInfo.obj
 0002:0000181c       $SG50638                   0040f81c     AccessInfo.obj
 0002:00001840       $SG50639                   0040f840     AccessInfo.obj
 0002:0000185c       $SG50640                   0040f85c     AccessInfo.obj
 0002:00001878       $SG50641                   0040f878     AccessInfo.obj
 0002:00001894       $SG50642                   0040f894     AccessInfo.obj
 0002:000018b0       $SG50643                   0040f8b0     AccessInfo.obj
 0002:000018cc       $SG50644                   0040f8cc     AccessInfo.obj
 0002:000018f4       $SG50647                   0040f8f4     AccessInfo.obj
 0002:00001914       $SG50648                   0040f914     AccessInfo.obj
 0002:0000193d       $SG71207                   0040f93d     MessageHistory.obj
 0002:0000193e       $SG71249                   0040f93e     MessageHistory.obj
 0002:0000193f       $SG71264                   0040f93f     MessageHistory.obj
 0002:00001940       $SG71271                   0040f940     MessageHistory.obj
 0002:00001941       $SG71309                   0040f941     MessageHistory.obj
 0002:00001942       $SG71323                   0040f942     MessageHistory.obj
 0002:00001943       $SG71325                   0040f943     MessageHistory.obj
 0002:00001968       ?jaccessinspectorOptionsRegistryKey@@3QBDB 0040f968     jaccessinspector.obj
 0002:0000196c       $SG50287                   0040f96c     jaccessinspector.obj
 0002:000019a4       $SG77725                   0040f9a4     jaccessinspector.obj
 0002:000019a8       $SG77726                   0040f9a8     jaccessinspector.obj
 0002:000019c0       $SG77727                   0040f9c0     jaccessinspector.obj
 0002:000019e4       $SG77728                   0040f9e4     jaccessinspector.obj
 0002:000019f8       $SG77794                   0040f9f8     jaccessinspector.obj
 0002:00001a14       $SG77802                   0040fa14     jaccessinspector.obj
 0002:00001a24       $SG77811                   0040fa24     jaccessinspector.obj
 0002:00001a34       $SG77906                   0040fa34     jaccessinspector.obj
 0002:00001a64       $SG77917                   0040fa64     jaccessinspector.obj
 0002:00001a98       $SG77928                   0040fa98     jaccessinspector.obj
 0002:00001ac8       $SG77939                   0040fac8     jaccessinspector.obj
 0002:00001af8       $SG77948                   0040faf8     jaccessinspector.obj
 0002:00001b14       $SG77956                   0040fb14     jaccessinspector.obj
 0002:00001b2c       $SG77966                   0040fb2c     jaccessinspector.obj
 0002:00001b68       $SG77975                   0040fb68     jaccessinspector.obj
 0002:00001b88       $SG77991                   0040fb88     jaccessinspector.obj
 0002:00001bc4       $SG77993                   0040fbc4     jaccessinspector.obj
 0002:00001be4       $SG77994                   0040fbe4     jaccessinspector.obj
 0002:00001bec       $SG77996                   0040fbec     jaccessinspector.obj
 0002:00001c0c       $SG77997                   0040fc0c     jaccessinspector.obj
 0002:00001c18       $SG78009                   0040fc18     jaccessinspector.obj
 0002:00001c60       $SG78020                   0040fc60     jaccessinspector.obj
 0002:00001c90       $SG78319                   0040fc90     jaccessinspector.obj
 0002:00001c9c       $SG78321                   0040fc9c     jaccessinspector.obj
 0002:00001cb0       $SG78323                   0040fcb0     jaccessinspector.obj
 0002:00001cc4       $SG78325                   0040fcc4     jaccessinspector.obj
 0002:00001cd8       $SG78327                   0040fcd8     jaccessinspector.obj
 0002:00001cec       $SG78329                   0040fcec     jaccessinspector.obj
 0002:00001cfc       $SG78331                   0040fcfc     jaccessinspector.obj
 0002:00001d08       $SG78333                   0040fd08     jaccessinspector.obj
 0002:00001d18       $SG78335                   0040fd18     jaccessinspector.obj
 0002:00001d24       $SG78337                   0040fd24     jaccessinspector.obj
 0002:00001d38       $SG78339                   0040fd38     jaccessinspector.obj
 0002:00001d4c       $SG78341                   0040fd4c     jaccessinspector.obj
 0002:00001d60       $SG78343                   0040fd60     jaccessinspector.obj
 0002:00001d74       $SG78345                   0040fd74     jaccessinspector.obj
 0002:00001d88       $SG78347                   0040fd88     jaccessinspector.obj
 0002:00001d9c       $SG78349                   0040fd9c     jaccessinspector.obj
 0002:00001db4       $SG78351                   0040fdb4     jaccessinspector.obj
 0002:00001dd4       $SG78353                   0040fdd4     jaccessinspector.obj
 0002:00001df0       $SG78355                   0040fdf0     jaccessinspector.obj
 0002:00001e0c       $SG78357                   0040fe0c     jaccessinspector.obj
 0002:00001e2c       $SG78359                   0040fe2c     jaccessinspector.obj
 0002:00001e44       $SG78361                   0040fe44     jaccessinspector.obj
 0002:00001e60       $SG78363                   0040fe60     jaccessinspector.obj
 0002:00001e80       $SG78365                   0040fe80     jaccessinspector.obj
 0002:00001e9c       $SG78367                   0040fe9c     jaccessinspector.obj
 0002:00001ec0       $SG78369                   0040fec0     jaccessinspector.obj
 0002:00001ee0       $SG78464                   0040fee0     jaccessinspector.obj
 0002:00001eec       $SG78467                   0040feec     jaccessinspector.obj
 0002:00001f00       $SG78470                   0040ff00     jaccessinspector.obj
 0002:00001f14       $SG78473                   0040ff14     jaccessinspector.obj
 0002:00001f28       $SG78476                   0040ff28     jaccessinspector.obj
 0002:00001f3c       $SG78479                   0040ff3c     jaccessinspector.obj
 0002:00001f4c       $SG78482                   0040ff4c     jaccessinspector.obj
 0002:00001f58       $SG78485                   0040ff58     jaccessinspector.obj
 0002:00001f68       $SG78488                   0040ff68     jaccessinspector.obj
 0002:00001f74       $SG78491                   0040ff74     jaccessinspector.obj
 0002:00001f88       $SG78494                   0040ff88     jaccessinspector.obj
 0002:00001f9c       $SG78497                   0040ff9c     jaccessinspector.obj
 0002:00001fb0       $SG78500                   0040ffb0     jaccessinspector.obj
 0002:00001fc4       $SG78503                   0040ffc4     jaccessinspector.obj
 0002:00001fd8       $SG78506                   0040ffd8     jaccessinspector.obj
 0002:00001fec       $SG78509                   0040ffec     jaccessinspector.obj
 0002:00002004       $SG78512                   00410004     jaccessinspector.obj
 0002:00002024       $SG78515                   00410024     jaccessinspector.obj
 0002:00002040       $SG78518                   00410040     jaccessinspector.obj
 0002:0000205c       $SG78521                   0041005c     jaccessinspector.obj
 0002:0000207c       $SG78524                   0041007c     jaccessinspector.obj
 0002:00002094       $SG78527                   00410094     jaccessinspector.obj
 0002:000020b0       $SG78530                   004100b0     jaccessinspector.obj
 0002:000020d0       $SG78533                   004100d0     jaccessinspector.obj
 0002:000020ec       $SG78536                   004100ec     jaccessinspector.obj
 0002:00002110       $SG78539                   00410110     jaccessinspector.obj
 0002:00002130       $SG78637                   00410130     jaccessinspector.obj
 0002:0000213c       _GS_ExceptionPointers      0041013c     MSVCRT:gs_report.obj
 0002:000028c8       __unwindtable$??0?$basic_string@DU?$char_traits@D@std@@V?$allocator@D@2@@std@@QAE@QBD@Z 004108c8     MessageHistory.obj
 0002:000028d0       __ehfuncinfo$??0?$basic_string@DU?$char_traits@D@std@@V?$allocator@D@2@@std@@QAE@QBD@Z 004108d0     MessageHistory.obj
 0002:000028f4       __ehfuncinfo$??1?$_List_alloc@U?$_List_base_types@V?$basic_string@DU?$char_traits@D@std@@V?$allocator@D@2@@std@@V?$allocator@V?$basic_string@DU?$char_traits@D@std@@V?$allocator@D@2@@std@@@2@@std@@@std@@QAE@XZ 004108f4     jaccessinspector.obj
 0002:000028f4       __ehfuncinfo$?__scrt_initialize_thread_safe_statics_platform_specific@@YAXXZ 004108f4     MSVCRT:thread_safe_statics.obj
 0002:000028f4       __ehfuncinfo$??1?$list@V?$basic_string@DU?$char_traits@D@std@@V?$allocator@D@2@@std@@V?$allocator@V?$basic_string@DU?$char_traits@D@std@@V?$allocator@D@2@@std@@@2@@std@@QAE@XZ 004108f4     jaccessinspector.obj
 0002:000028f4       __ehfuncinfo$?clear@?$list@V?$basic_string@DU?$char_traits@D@std@@V?$allocator@D@2@@std@@V?$allocator@V?$basic_string@DU?$char_traits@D@std@@V?$allocator@D@2@@std@@@2@@std@@QAEXXZ 004108f4     MessageHistory.obj
 0002:000028f4       __ehfuncinfo$?_Make_iter@?$list@V?$basic_string@DU?$char_traits@D@std@@V?$allocator@D@2@@std@@V?$allocator@V?$basic_string@DU?$char_traits@D@std@@V?$allocator@D@2@@std@@@2@@std@@QBE?AV?$_List_iterator@V?$_List_val@U?$_List_simple_types@V?$basic_string@DU?$char_traits@D@std@@V?$allocator@D@2@@std@@@std@@@std@@@2@V?$_List_const_iterator@V?$_List_val@U?$_List_simple_types@V?$basic_string@DU?$char_traits@D@std@@V?$allocator@D@2@@std@@@std@@@std@@@2@@Z 004108f4     MessageHistory.obj
 0002:000028f4       __ehfuncinfo$?end@?$list@V?$basic_string@DU?$char_traits@D@std@@V?$allocator@D@2@@std@@V?$allocator@V?$basic_string@DU?$char_traits@D@std@@V?$allocator@D@2@@std@@@2@@std@@QAE?AV?$_List_iterator@V?$_List_val@U?$_List_simple_types@V?$basic_string@DU?$char_traits@D@std@@V?$allocator@D@2@@std@@@std@@@std@@@2@XZ 004108f4     MessageHistory.obj
 0002:000028f4       __ehfuncinfo$?begin@?$list@V?$basic_string@DU?$char_traits@D@std@@V?$allocator@D@2@@std@@V?$allocator@V?$basic_string@DU?$char_traits@D@std@@V?$allocator@D@2@@std@@@2@@std@@QAE?AV?$_List_iterator@V?$_List_val@U?$_List_simple_types@V?$basic_string@DU?$char_traits@D@std@@V?$allocator@D@2@@std@@@std@@@std@@@2@XZ 004108f4     MessageHistory.obj
 0002:000028f4       __ehfuncinfo$?c_str@?$basic_string@DU?$char_traits@D@std@@V?$allocator@D@2@@std@@QBEPBDXZ 004108f4     MessageHistory.obj
 0002:000028f4       __ehfuncinfo$??1?$basic_string@DU?$char_traits@D@std@@V?$allocator@D@2@@std@@QAE@XZ 004108f4     MessageHistory.obj
 0002:000028f4       __ehfuncinfo$?_Assign_rv_contents_with_alloc_always_equal@?$basic_string@DU?$char_traits@D@std@@V?$allocator@D@2@@std@@QAEX$$QAV12@U?$integral_constant@_N$00@2@@Z 004108f4     MessageHistory.obj
 0002:000028f4       __ehfuncinfo$??0?$basic_string@DU?$char_traits@D@std@@V?$allocator@D@2@@std@@QAE@$$QAV01@@Z 004108f4     MessageHistory.obj
 0002:000028f4       __ehfuncinfo$??$_Freenode0@V?$allocator@U?$_List_node@V?$basic_string@DU?$char_traits@D@std@@V?$allocator@D@2@@std@@PAX@std@@@std@@@?$_List_node@V?$basic_string@DU?$char_traits@D@std@@V?$allocator@D@2@@std@@PAX@std@@SAXAAV?$allocator@U?$_List_node@V?$basic_string@DU?$char_traits@D@std@@V?$allocator@D@2@@std@@PAX@std@@@1@PAU01@@Z 004108f4     MessageHistory.obj
 0002:00002918       __catchsym$?_Buynode0@?$_List_alloc@U?$_List_base_types@V?$basic_string@DU?$char_traits@D@std@@V?$allocator@D@2@@std@@V?$allocator@V?$basic_string@DU?$char_traits@D@std@@V?$allocator@D@2@@std@@@2@@std@@@std@@QAEPAU?$_List_node@V?$basic_string@DU?$char_traits@D@std@@V?$allocator@D@2@@std@@PAX@2@PAU32@0@Z$2 00410918     MessageHistory.obj
 0002:00002928       __unwindtable$?_Buynode0@?$_List_alloc@U?$_List_base_types@V?$basic_string@DU?$char_traits@D@std@@V?$allocator@D@2@@std@@V?$allocator@V?$basic_string@DU?$char_traits@D@std@@V?$allocator@D@2@@std@@@2@@std@@@std@@QAEPAU?$_List_node@V?$basic_string@DU?$char_traits@D@std@@V?$allocator@D@2@@std@@PAX@2@PAU32@0@Z 00410928     MessageHistory.obj
 0002:00002938       __tryblocktable$?_Buynode0@?$_List_alloc@U?$_List_base_types@V?$basic_string@DU?$char_traits@D@std@@V?$allocator@D@2@@std@@V?$allocator@V?$basic_string@DU?$char_traits@D@std@@V?$allocator@D@2@@std@@@2@@std@@@std@@QAEPAU?$_List_node@V?$basic_string@DU?$char_traits@D@std@@V?$allocator@D@2@@std@@PAX@2@PAU32@0@Z 00410938     MessageHistory.obj
 0002:0000294c       __ehfuncinfo$?_Buynode0@?$_List_alloc@U?$_List_base_types@V?$basic_string@DU?$char_traits@D@std@@V?$allocator@D@2@@std@@V?$allocator@V?$basic_string@DU?$char_traits@D@std@@V?$allocator@D@2@@std@@@2@@std@@@std@@QAEPAU?$_List_node@V?$basic_string@DU?$char_traits@D@std@@V?$allocator@D@2@@std@@PAX@2@PAU32@0@Z 0041094c     MessageHistory.obj
 0002:00002970       __unwindtable$?AddMessage@MessageHistory@@QAEXPBD@Z 00410970     MessageHistory.obj
 0002:00002978       __ehfuncinfo$?AddMessage@MessageHistory@@QAEXPBD@Z 00410978     MessageHistory.obj
 0002:0000299c       __catchsym$??$_Buynode@V?$basic_string@DU?$char_traits@D@std@@V?$allocator@D@2@@std@@@?$_List_buy@V?$basic_string@DU?$char_traits@D@std@@V?$allocator@D@2@@std@@V?$allocator@V?$basic_string@DU?$char_traits@D@std@@V?$allocator@D@2@@std@@@2@@std@@QAEPAU?$_List_node@V?$basic_string@DU?$char_traits@D@std@@V?$allocator@D@2@@std@@PAX@1@PAU21@0$$QAV?$basic_string@DU?$char_traits@D@std@@V?$allocator@D@2@@1@@Z$2 0041099c     MessageHistory.obj
 0002:000029ac       __unwindtable$??$_Buynode@V?$basic_string@DU?$char_traits@D@std@@V?$allocator@D@2@@std@@@?$_List_buy@V?$basic_string@DU?$char_traits@D@std@@V?$allocator@D@2@@std@@V?$allocator@V?$basic_string@DU?$char_traits@D@std@@V?$allocator@D@2@@std@@@2@@std@@QAEPAU?$_List_node@V?$basic_string@DU?$char_traits@D@std@@V?$allocator@D@2@@std@@PAX@1@PAU21@0$$QAV?$basic_string@DU?$char_traits@D@std@@V?$allocator@D@2@@1@@Z 004109ac     MessageHistory.obj
 0002:000029bc       __tryblocktable$??$_Buynode@V?$basic_string@DU?$char_traits@D@std@@V?$allocator@D@2@@std@@@?$_List_buy@V?$basic_string@DU?$char_traits@D@std@@V?$allocator@D@2@@std@@V?$allocator@V?$basic_string@DU?$char_traits@D@std@@V?$allocator@D@2@@std@@@2@@std@@QAEPAU?$_List_node@V?$basic_string@DU?$char_traits@D@std@@V?$allocator@D@2@@std@@PAX@1@PAU21@0$$QAV?$basic_string@DU?$char_traits@D@std@@V?$allocator@D@2@@1@@Z 004109bc     MessageHistory.obj
 0002:000029d0       __ehfuncinfo$??$_Buynode@V?$basic_string@DU?$char_traits@D@std@@V?$allocator@D@2@@std@@@?$_List_buy@V?$basic_string@DU?$char_traits@D@std@@V?$allocator@D@2@@std@@V?$allocator@V?$basic_string@DU?$char_traits@D@std@@V?$allocator@D@2@@std@@@2@@std@@QAEPAU?$_List_node@V?$basic_string@DU?$char_traits@D@std@@V?$allocator@D@2@@std@@PAX@1@PAU21@0$$QAV?$basic_string@DU?$char_traits@D@std@@V?$allocator@D@2@@1@@Z 004109d0     MessageHistory.obj
 0002:000029f4       __unwindtable$??0MessageHistory@@QAE@XZ 004109f4     jaccessinspector.obj
 0002:000029fc       __ehfuncinfo$??0MessageHistory@@QAE@XZ 004109fc     jaccessinspector.obj
 0002:00002a20       __sehtable$___scrt_is_nonwritable_in_current_image 00410a20     MSVCRT:utility.obj
 0002:00002a40       __sehtable$?__scrt_common_main_seh@@YAHXZ 00410a40     MSVCRT:exe_winmain.obj
 0002:00002e88       .idata$6                   00410e88     advapi32:ADVAPI32.dll
 0002:00003128       .idata$6                   00411128     user32:USER32.dll
 0002:00003154       .idata$6                   00411154     msvcprt:MSVCP140.dll
 0002:000033a2       .idata$6                   004113a2     kernel32:KERNEL32.dll
 0002:00003446       .idata$6                   00411446     vcruntime:VCRUNTIME140.dll
 0002:00003718       .idata$6                   00411718     ucrt:api-ms-win-crt-string-l1-1-0.dll
 0002:0000373a       .idata$6                   0041173a     ucrt:api-ms-win-crt-stdio-l1-1-0.dll
 0002:0000375a       .idata$6                   0041175a     ucrt:api-ms-win-crt-environment-l1-1-0.dll
 0002:00003780       .idata$6                   00411780     ucrt:api-ms-win-crt-time-l1-1-0.dll
 0002:000037a0       .idata$6                   004117a0     ucrt:api-ms-win-crt-runtime-l1-1-0.dll
 0002:000037c2       .idata$6                   004117c2     ucrt:api-ms-win-crt-heap-l1-1-0.dll
 0002:000037e2       .idata$6                   004117e2     ucrt:api-ms-win-crt-math-l1-1-0.dll
 0002:00003802       .idata$6                   00411802     ucrt:api-ms-win-crt-locale-l1-1-0.dll
 0003:00000000       $SG46583                   00412000     AccessBridgeCalls.obj
 0003:00000018       $SG46587                   00412018     AccessBridgeCalls.obj
 0003:00000024       $SG46589                   00412024     AccessBridgeCalls.obj
 0003:00000038       $SG46591                   00412038     AccessBridgeCalls.obj
 0003:0000004c       $SG46593                   0041204c     AccessBridgeCalls.obj
 0003:0000005c       $SG46595                   0041205c     AccessBridgeCalls.obj
 0003:00000070       $SG46597                   00412070     AccessBridgeCalls.obj
 0003:00000084       $SG46599                   00412084     AccessBridgeCalls.obj
 0003:00000098       $SG46601                   00412098     AccessBridgeCalls.obj
 0003:000000ac       $SG46603                   004120ac     AccessBridgeCalls.obj
 0003:000000c0       $SG46605                   004120c0     AccessBridgeCalls.obj
 0003:000000d4       $SG46607                   004120d4     AccessBridgeCalls.obj
 0003:000000e8       $SG46609                   004120e8     AccessBridgeCalls.obj
 0003:000000fc       $SG46611                   004120fc     AccessBridgeCalls.obj
 0003:00000110       $SG46613                   00412110     AccessBridgeCalls.obj
 0003:00000128       $SG46615                   00412128     AccessBridgeCalls.obj
 0003:0000014c       $SG46617                   0041214c     AccessBridgeCalls.obj
 0003:0000016c       $SG46619                   0041216c     AccessBridgeCalls.obj
 0003:00000184       $SG46621                   00412184     AccessBridgeCalls.obj
 0003:000001a4       $SG46623                   004121a4     AccessBridgeCalls.obj
 0003:000001c0       $SG46625                   004121c0     AccessBridgeCalls.obj
 0003:000001dc       $SG46627                   004121dc     AccessBridgeCalls.obj
 0003:000001fc       $SG46629                   004121fc     AccessBridgeCalls.obj
 0003:00000214       $SG46631                   00412214     AccessBridgeCalls.obj
 0003:00000230       $SG46633                   00412230     AccessBridgeCalls.obj
 0003:00000250       $SG46635                   00412250     AccessBridgeCalls.obj
 0003:0000026c       $SG46637                   0041226c     AccessBridgeCalls.obj
 0003:00000290       $SG46639                   00412290     AccessBridgeCalls.obj
 0003:000002b0       $SG46641                   004122b0     AccessBridgeCalls.obj
 0003:000002c4       $SG46643                   004122c4     AccessBridgeCalls.obj
 0003:000002d4       $SG46645                   004122d4     AccessBridgeCalls.obj
 0003:000002e4       $SG46647                   004122e4     AccessBridgeCalls.obj
 0003:000002f4       $SG46649                   004122f4     AccessBridgeCalls.obj
 0003:00000314       $SG46651                   00412314     AccessBridgeCalls.obj
 0003:00000334       $SG46653                   00412334     AccessBridgeCalls.obj
 0003:0000034c       $SG46655                   0041234c     AccessBridgeCalls.obj
 0003:0000036c       $SG46657                   0041236c     AccessBridgeCalls.obj
 0003:00000388       $SG46659                   00412388     AccessBridgeCalls.obj
 0003:000003a8       $SG46661                   004123a8     AccessBridgeCalls.obj
 0003:000003c8       $SG46663                   004123c8     AccessBridgeCalls.obj
 0003:000003e0       $SG46665                   004123e0     AccessBridgeCalls.obj
 0003:000003fc       $SG46667                   004123fc     AccessBridgeCalls.obj
 0003:00000418       $SG46669                   00412418     AccessBridgeCalls.obj
 0003:00000438       $SG46671                   00412438     AccessBridgeCalls.obj
 0003:0000045c       $SG46673                   0041245c     AccessBridgeCalls.obj
 0003:00000480       $SG46675                   00412480     AccessBridgeCalls.obj
 0003:000004a4       $SG46677                   004124a4     AccessBridgeCalls.obj
 0003:000004c4       $SG46679                   004124c4     AccessBridgeCalls.obj
 0003:000004e4       $SG46681                   004124e4     AccessBridgeCalls.obj
 0003:0000050c       $SG46683                   0041250c     AccessBridgeCalls.obj
 0003:0000052c       $SG46685                   0041252c     AccessBridgeCalls.obj
 0003:00000550       $SG46687                   00412550     AccessBridgeCalls.obj
 0003:00000568       $SG46689                   00412568     AccessBridgeCalls.obj
 0003:00000584       $SG46691                   00412584     AccessBridgeCalls.obj
 0003:0000059c       $SG46693                   0041259c     AccessBridgeCalls.obj
 0003:000005b8       $SG46695                   004125b8     AccessBridgeCalls.obj
 0003:000005d0       $SG46697                   004125d0     AccessBridgeCalls.obj
 0003:000005ec       $SG46699                   004125ec     AccessBridgeCalls.obj
 0003:00000608       $SG46701                   00412608     AccessBridgeCalls.obj
 0003:00000624       $SG46703                   00412624     AccessBridgeCalls.obj
 0003:00000644       $SG46705                   00412644     AccessBridgeCalls.obj
 0003:0000065c       $SG46707                   0041265c     AccessBridgeCalls.obj
 0003:00000678       $SG46709                   00412678     AccessBridgeCalls.obj
 0003:0000068c       $SG46711                   0041268c     AccessBridgeCalls.obj
 0003:000006a4       $SG46713                   004126a4     AccessBridgeCalls.obj
 0003:000006b8       $SG46715                   004126b8     AccessBridgeCalls.obj
 0003:000006d0       $SG46717                   004126d0     AccessBridgeCalls.obj
 0003:000006e8       $SG46719                   004126e8     AccessBridgeCalls.obj
 0003:00000708       $SG46721                   00412708     AccessBridgeCalls.obj
 0003:00000724       $SG46723                   00412724     AccessBridgeCalls.obj
 0003:0000073c       $SG46725                   0041273c     AccessBridgeCalls.obj
 0003:00000758       $SG46727                   00412758     AccessBridgeCalls.obj
 0003:00000770       $SG46729                   00412770     AccessBridgeCalls.obj
 0003:00000798       $SG46731                   00412798     AccessBridgeCalls.obj
 0003:000007c0       $SG46733                   004127c0     AccessBridgeCalls.obj
 0003:000007e8       $SG46735                   004127e8     AccessBridgeCalls.obj
 0003:0000080c       $SG46737                   0041280c     AccessBridgeCalls.obj
 0003:00000830       $SG46739                   00412830     AccessBridgeCalls.obj
 0003:00000854       $SG46741                   00412854     AccessBridgeCalls.obj
 0003:0000087c       $SG46743                   0041287c     AccessBridgeCalls.obj
 0003:000008a4       $SG46745                   004128a4     AccessBridgeCalls.obj
 0003:000008cc       $SG46747                   004128cc     AccessBridgeCalls.obj
 0003:000008f4       $SG46749                   004128f4     AccessBridgeCalls.obj
 0003:00000904       $SG46751                   00412904     AccessBridgeCalls.obj
 0003:00000918       $SG46753                   00412918     AccessBridgeCalls.obj
 0003:0000092c       $SG46755                   0041292c     AccessBridgeCalls.obj
 0003:00000948       $SG46757                   00412948     AccessBridgeCalls.obj
 0003:00000958       $SG46759                   00412958     AccessBridgeCalls.obj
 0003:0000096c       $SG46761                   0041296c     AccessBridgeCalls.obj
 0003:00000988       $SG46763                   00412988     AccessBridgeCalls.obj
 0003:00000998       $SG46765                   00412998     AccessBridgeCalls.obj
 0003:000009a8       $SG46767                   004129a8     AccessBridgeCalls.obj
 0003:000009c4       $SG46769                   004129c4     AccessBridgeCalls.obj
 0003:000009dc       $SG46771                   004129dc     AccessBridgeCalls.obj
 0003:000009f0       $SG46773                   004129f0     AccessBridgeCalls.obj
 0003:00000a04       $SG46775                   00412a04     AccessBridgeCalls.obj
 0003:00000a18       $SG46777                   00412a18     AccessBridgeCalls.obj
 0003:00000a2c       ?warning@?1??appendToBuffer@@YAHPADI0ZZ@4PADA 00412a2c     AccessInfo.obj
 0003:00000b50       _logFP                     00412b50     AccessBridgeDebug.obj
 0003:00000b58       ?retbuf@?1??printError@@9@4PADA 00412b58     AccessBridgeDebug.obj
 0003:00000c68       ?datebuf@?1??getTimeAndDate@@YAPADXZ@4PADA 00412c68     AccessInfo.obj
 0003:00000d44       ?titleBarHeight@?1??jaccessinspectorDialogProc@@YGHPAUHWND__@@IIJ@Z@4HA 00412d44     jaccessinspector.obj
 0003:00000d48       ?$TSS0@?1??jaccessinspectorDialogProc@@YGHPAUHWND__@@IIJ@Z@4HA 00412d48     jaccessinspector.obj
 0003:00000d4c       ?menuBarHeight@?1??jaccessinspectorDialogProc@@YGHPAUHWND__@@IIJ@Z@4HA 00412d4c     jaccessinspector.obj
 0003:00000d50       ?$TSS1@?1??jaccessinspectorDialogProc@@YGHPAUHWND__@@IIJ@Z@4HA 00412d50     jaccessinspector.obj
 0003:00000d54       ?borderHeight@?1??jaccessinspectorDialogProc@@YGHPAUHWND__@@IIJ@Z@4HA 00412d54     jaccessinspector.obj
 0003:00000d58       ?$TSS2@?1??jaccessinspectorDialogProc@@YGHPAUHWND__@@IIJ@Z@4HA 00412d58     jaccessinspector.obj
 0003:00000d5c       ?borderWidth@?1??jaccessinspectorDialogProc@@YGHPAUHWND__@@IIJ@Z@4HA 00412d5c     jaccessinspector.obj
 0003:00000d60       ?$TSS3@?1??jaccessinspectorDialogProc@@YGHPAUHWND__@@IIJ@Z@4HA 00412d60     jaccessinspector.obj
 0003:00000d64       ?verticalScrollBarWidth@?1??jaccessinspectorDialogProc@@YGHPAUHWND__@@IIJ@Z@4HA 00412d64     jaccessinspector.obj
 0003:00000d68       ?$TSS4@?1??jaccessinspectorDialogProc@@YGHPAUHWND__@@IIJ@Z@4HA 00412d68     jaccessinspector.obj
 0003:00000d70       _GS_ExceptionRecord        00412d70     MSVCRT:gs_report.obj
 0003:00000dc0       _GS_ContextRecord          00412dc0     MSVCRT:gs_report.obj
 0003:00001094       ?is_initialized_as_dll@@3_NA 00413094     MSVCRT:utility.obj
 0003:00001095       ?module_local_atexit_table_initialized@@3_NA 00413095     MSVCRT:utility.obj
 0003:00001098       ?module_local_atexit_table@@3U_onexit_table_t@@A 00413098     MSVCRT:utility.obj
 0003:000010a4       ?module_local_at_quick_exit_table@@3U_onexit_table_t@@A 004130a4     MSVCRT:utility.obj
 0003:000010b0       ?_Tss_mutex@@3U_RTL_CRITICAL_SECTION@@A 004130b0     MSVCRT:thread_safe_statics.obj
 0003:000010c8       ?_Tss_cv@@3U_RTL_CONDITION_VARIABLE@@A 004130c8     MSVCRT:thread_safe_statics.obj
 0003:000010cc       ?_Tss_event@@3PAXA         004130cc     MSVCRT:thread_safe_statics.obj
 0003:000010d0       ?encoded_sleep_condition_variable_cs@@3P6GHPAU_RTL_CONDITION_VARIABLE@@PAU_RTL_CRITICAL_SECTION@@K@ZA 004130d0     MSVCRT:thread_safe_statics.obj
 0003:000010d4       ?encoded_wake_all_condition_variable@@3P6GXPAU_RTL_CONDITION_VARIABLE@@@ZA 004130d4     MSVCRT:thread_safe_statics.obj
 0004:000001c0       $R000000                   004141c0     jaccessinspector-32.exe.res
 0004:00000358       $R000198                   00414358     jaccessinspector-32.exe.res
 0004:00000468       $R0002A8                   00414468     jaccessinspector-32.exe.res
 0004:00000d10       $R000B50                   00414d10     jaccessinspector-32.exe.res
 0004:00001050       $R000E90                   00415050     jaccessinspector-32.exe.res
